:100000000C94B1070C94D9070C94D9070C94D90718
:100010000C94D9070C94D9070C94D9070C94D907E0
:100020000C94D9070C94D9070C9477190C94E61901
:100030000C94D9070C94D9070C94D9070C94D907C0
:100040000C94D9070C94D9070C94D9070C94D907B0
:100050000C94D9070C94D9070C94D9070C94181C4C
:100060000C94D9070C94D9070C94D9070C94D90790
:100070000C94D9070C94D9070C94D9070C94D90780
:100080000C94D9070C94D9070C94D9070C94D90770
:100090000C94D9070C94D9070C94D9070C94D90760
:1000A0000C94D9070C94D9070C94D90744617900B2
:1000B00041636374004C6F616E00436170616369FA
:1000C0007479200053707261792000050512151FA4
:1000D000150905082466E766244120596573202028
:1000E00042204E6F000043616E6479204361737457
:1000F0006C6500536F6461205377616D70004775C4
:100100006D6D7920466F726573740043686F636F1D
:100110006C616E640049636520437265616D2052B5
:1001200064005377656574205375697465730000C6
:100130004C6F6C6C7900536F757273004D61727304
:10014000004165726F004865727368657900502ED2
:100150005375676172002000200003081F051F1FF0
:10016000151B1F11111F110E1F15111F05011F1146
:100170001D1F041F001F0010101F1F041B1F101045
:100180001F061F1F011F1F111F1F05071F311F1FE4
:10019000051B17151D011F011F101F0F100F1F0C2E
:1001A0001F1B041B071C071915130C121E1F120C12
:1001B0001E12120C121F0C1A14041F052E2A1E1FC9
:1001C000021C001D00201D001F041A011F001E0438
:1001D0001E1E021E1E121E3E120C0C123E1E020697
:1001E00014120A020F121E101E0E100E1E081E1AE6
:1001F000041A2E281E1A12161F111F001F001D158B
:100200001711151F07041F17151D1F151D01011FAD
:100210001F151F17151F00170000100020100000E9
:10022000030004083E09093E3F25251A1E2121121C
:100230003F21211E3F2525213F0505011E21293A89
:100240003F04043F213F21001021211F3F040A31B8
:100250003F2020203F02023F3F02043F1E21211E7B
:100260003F0909061E21112E3F09093622252519AD
:10027000013F01011F20201F0F10201F3F10103FC2
:100280003B04043B03043807312D2321102A2A3C68
:100290003F2424181C2222141824243F1C2A2A2C10
:1002A000047E05014C52523E3F040438243D200098
:1002B0004040443D3F081422213F20003E04043EBC
:1002C0003E04023C1C22221C7E22221C1C22227E76
:1002D0003E040204242A2A12021F22201E20201E6D
:1002E0000E10201E3E10103E360808364E50503E6E
:1002F000322A26221E29251E223F200032292926A5
:100300001221251A0C0A3F08172525191E25251824
:10031000013905031A25251A0629291E002F000078
:10032000002000004020000000030000000000004A
:10033000003E5B4F5B3E3E6B4F6B3E1C3E7C3E1C6B
:10034000183C7E3C181C577D571C1C5E7F5E1C00B1
:10035000183C1800FFE7C3E7FF0018241800FFE768
:10036000DBE7FF30483A060E2629792926407F052B
:100370000507407F05253F5A3CE73C5A7F3E1C1C41
:1003800008081C1C3E7F14227F22145F5F005F5F01
:1003900006097F017F006689956A606060606094ED
:1003A000A2FFA29408047E040810207E20100808F2
:1003B0002A1C08081C2A08081E101010100C1E0CFD
:1003C0001E0C30383E3830060E3E0E06000000008F
:1003D0000000005F00000007000700147F147F1476
:1003E000242A7F2A122313086462364956205000BB
:1003F00008070300001C2241000041221C002A1CA7
:100400007F1C2A08083E0808008070300008080891
:100410000808000060600020100804023E514945B1
:100420003E00427F400072494949462141494D33CF
:100430001814127F1027454545393C4A4949314136
:10044000211109073649494936464949291E000004
:100450001400000040340000000814224114141459
:100460001414004122140802015909063E415D5945
:100470004E7C1211127C7F494949363E414141224E
:100480007F4141413E7F494949417F090909013E78
:10049000414151737F0808087F00417F410020409F
:1004A000413F017F081422417F404040407F021CB1
:1004B000027F7F0408107F3E4141413E7F090909C8
:1004C000063E4151215E7F09192946264949493294
:1004D00003017F01033F4040403F1F2040201F3F5A
:1004E0004038403F631408146303047804036159DF
:1004F000494D43007F414141020408102000414121
:10050000417F0402010204404040404000030708CC
:100510000020545478407F284444383844444428C8
:10052000384444287F385454541800087E0902186F
:10053000A4A49C787F0804047800447D40002040F7
:10054000403D007F1028440000417F40007C04783B
:1005500004787C080404783844444438FC18242483
:100560001818242418FC7C08040408485454542403
:1005700004043F44243C4040207C1C2040201C3C80
:100580004030403C44281028444C9090907C446477
:10059000544C44000836410000007700000041360A
:1005A000080002010204023C2623263C1EA1A16190
:1005B000123A4040207A38545455592155557941C2
:1005C0002154547841215554784020545579400C99
:1005D0001E5272123955555559395454545939557A
:1005E0005454580000457C410002457D42000145BD
:1005F0007C40F0292429F0F0282528F07C5455452A
:10060000002054547C547C0A097F493249494932BC
:100610003248484832324A4848303A4141217A3AD1
:1006200042402078009DA0A07D39444444393D409B
:1006300040403D3C24FF2424487E4943662B2FFC48
:100640002F2BFF0929F620C0887E090320545479F6
:10065000410000447D413048484A32384040227AC7
:10066000007A0A0A727D0D19317D2629292F282644
:100670002929292630484D4020380808080808084C
:100680000808382F10C8ACBA2F102834FA00007BA5
:10069000000008142A142222142A140895002200AB
:1006A00095AA005500AAAA55AA55AA000000FF0065
:1006B000101010FF00141414FF001010FF00FF10A2
:1006C00010F010F0141414FC001414F700FF0000D4
:1006D000FF00FF1414F404FC141417101F10101F53
:1006E000101F1414141F00101010F0000000001F41
:1006F000101010101F10101010F010000000FF104C
:100700001010101010101010FF10000000FF140047
:1007100000FF00FF00001F10170000FC04F4141479
:100720001710171414F404F40000FF00F714141445
:1007300014141414F700F7141414171410101F10C5
:100740001F141414F4141010F010F000001F101FE8
:100750000000001F14000000FC140000F010F01056
:1007600010FF10FF141414FF141010101F000000CD
:1007700000F010FFFFFFFFFFF0F0F0F0F0FFFFFFD1
:100780000000000000FFFF0F0F0F0F0F3844443828
:10079000447C2A2A3E147E02020606027E027E0263
:1007A00063554941633844443C04407E201E200682
:1007B000027E020299A5E7A5991C2A492A1C4C72BF
:1007C00001724C304A4D4D303048784830BC625A46
:1007D000463D3E494949007E0101017E2A2A2A2AD6
:1007E0002A44445F444440514A444040444A5140B2
:1007F0000000FF0103E080FF000008086B6B083673
:1008000012362436060F090F0600001818000000E3
:100810001010003040FF0101001F01011E00191DD2
:100820001712003C3C3C3C0000000000D5F08D1449
:10083000A1C881CFD9F1AF2000F0F89C8E878387C3
:100840008E9CF8F00000FEFF0303030303070EFC79
:10085000F80000FEFF0303030303070EFCF800008B
:10086000FFFF00000000000000FFFF0000FEFF830C
:1008700083838383C7EE7C380000F8FC0E070303F4
:1008800003070EFCF800003F7FE0C08080C0E07FDF
:100890003FFFFF01010101010101FFFF0000FFFF18
:1008A0000C0C0C0C1C3E77E3C100007FFFC0C0C0E5
:1008B000C0C0E0703F1F00001F3F70E0C0C0C0E03C
:1008C000703F1F00007FFFC1C1C1C1C1E3773E1C63
:1008D00000001F3F70E0C0C0C0E0703F1F0000007C
:1008E000000001FFFF01000000647572696E67205F
:1008F0007468652063686173652121006275636BAC
:10090000732066726F6D2070757273657300596F16
:100910007520736E6174636865642000546865793E
:1009200020616C6C20676176652075702100412024
:100930004D6F6D2067617665207570212100002064
:1009400020596F75206D6973736564212121000042
:100950006861766520746F2072756E2100616E7912
:100960002073707261792120596F7500596F75205D
:10097000646F6E27742068617665007468656D2108
:1009800000596F752063616E2774207368616B6511
:1009900000616E20616C6C6579212100596F7520B2
:1009A0006C6F7374207468656D20696E00756E6974
:1009B0007473206F663A2000596F7520666F756EEC
:1009C000642000323030206275636B733F006D6FBE
:1009D000726520737061636520666F720063616E7B
:1009E0006479207361636B20776974680057696C60
:1009F0006C20796F75206275792061206E657700B3
:100A000057696C6C20796F75206561742069743F3B
:100A1000006D6F73746C7920756E636865776564BB
:100A2000212100686572652074686174206C6F6FA5
:100A30006B73005468657265277320736F6D652052
:100A400067756D00646F6C6C6172733F00737072D8
:100A5000617920666F7220343030004D6F6D2072E6
:100A60006570656C6C616E74007374696E6B207375
:100A70007072617920666F7200736C6565702073A7
:100A80007072617920666F720034303020646F6C50
:100A90006C6172733F0057696C6C20796F752062CE
:100AA0007579206100616674657220796F75210027
:100AB000667269656E64732061726500206F6620DE
:100AC00068657200616E642000596F7572204D6F09
:100AD0007468657200746F2063686172697479214B
:100AE00000596F7520676176652061206269740026
:100AF000617265206F7574726167656F757321210E
:100B000021210073686F72746167652120507269DA
:100B100063657300506F77646572656420737567F1
:100B20006172007072696365732121210061742014
:100B30006F7574726167656F757300627579696E40
:100B40006720486572736865790043686F636F68F2
:100B50006F6C696373206172650062616B652D6FF4
:100B60006666212121210066726F6D206C617374AD
:100B7000207765656B277300636865617020486541
:100B80007273686579004D6F6D73206172652073B3
:100B9000656C6C696E6700626F74746F6D6564205C
:100BA0006F7574212121004D617273207072696329
:100BB00065732068617665006C6F6C6C792121210A
:100BC000006172652073656C6C696E67206368658F
:100BD0006170004B696473206174207363686F6F88
:100BE0006C00746F6461792100626F72726F776557
:100BF00064206D6F6E657900596F7520616C726548
:100C0000616479002100596F7520646F6E2774202C
:100C10006861766520616E7900004F6F7073210006
:100C20002100596F752063616E2774206166666FBD
:100C3000726400004F6F7073210021006D6F726548
:100C40002000596F752063616E2774206361727292
:100C50007900004F6F70732100596F7527726520FE
:100C60006361756768742121006265656E2068693B
:100C7000742100596F75277665006D69737365641B
:100C80002121005468657900796F75212120005475
:100C9000686579277265206E616767696E670041D4
:100CA0002053707261792020422052756E004552A7
:100CB000524F522000416D7400536176696E677324
:100CC00000596F75206F776500596F7520686176E0
:100CD00065005769746864726177204D6F6E65793D
:100CE000004465706F736974204D6F6E65790042C2
:100CF0006F72726F77204D6F6E6579005061792049
:100D00004C6F616E00000051747900507269636528
:100D100000436F73747300596F75206861766500C6
:100D200053656C6C200042757920000000796F7566
:100D3000722074656574683F0064656E74697374CD
:100D400020746F2066697800646F6C6C6172732028
:100D5000666F7220610057696C6C20796F75207026
:100D60006179203130303000596F757220686561CB
:100D70006C74683A20007374696C6C2061667465E9
:100D80007220796F752100204D6F6D730054686576
:100D900072652061726520004265696E6720636834
:100DA00061736564212100576974686472617720FA
:100DB0004D6F6E6579004465706F736974204D6F77
:100DC0006E65790042616E6B00426F72726F7720C0
:100DD0004D6F6E6579005265706179204C6F616E60
:100DE0000052696368204275646479004A65742022
:100DF00066726F6D200053656C6C2043616E647980
:100E0000004275792043616E64790043616E6479B4
:100E1000205361636B0042616E6B0052696368200E
:100E20004275646479004A65740043616E64792098
:100E30005361636B0053656C6C2043616E64790091
:100E40004275792043616E64790048697420746842
:100E500065205374726565747321210076312E30DC
:100E60000043616E6479576172001E1E000000002D
:100E7000000000000000000000C0F0E8C48202038F
:100E80003F3F0F8782C2C4C8F0C0000000000000CE
:100E9000008080807088A80FF1810181C1E1F0FCA1
:100EA000F000818143271F0700000000008040A15F
:100EB000562C1434224176080D0907010101010165
:100EC0000000000000003028140A050201000000A4
:100ED0000000000000000000000000000000000012
:100EE00000000000080B00020202000009040000DC
:100EF0000102020000052400100105240101010483
:100F0000240206052406000107058103100040099C
:100F1000040100020A000000070502024000000769
:100F20000583024000000403090412010002EF02DD
:100F300001404123368000010102030141726475C2
:100F4000696E6F204C4C430041726475696E6F206E
:100F50004C656F6E6172646F0003051F0E04951C73
:100F6000D62E11241FBECFEFDAE0DEBFCDBF12E0D8
:100F7000A0E0B1E0ECE6FBE602C005900D92A635DC
:100F8000B107D9F727E0A6E5B2E001C01D92A03A6B
:100F9000B207E1F717E0C0EBD7E004C02197FE01EC
:100FA0000E94B133CF3AD107C9F70E94161D0C94A5
:100FB000A9350C940000E6EEF2E0A0E0B8E0008075
:100FC0000EBC8111012C1197A0FDFDCF0192B9F744
:100FD0000DB40895480F592F511D1416150684F5A8
:100FE000803891056CF597FF02C090E080E04138B1
:100FF000510514F040E850E0481BFB01E770FF2763
:1010000021E001C0220FEA95EAF777FF02C0695F8D
:101010007F4FFB0133E0F595E7953A95E1F7F695BB
:10102000FE2FEE27F795E795E80FF91FEA51FD4FE0
:10103000415030F08191DF011197822B8C93F8CFD2
:1010400008956F927F928F929F92AF92BF92CF92AC
:10105000DF92EF92FF920F931F93CF93DF93DC0108
:10106000FA011491319654913196C12FD0E0222388
:1010700009F1CC24C394D12C852F877011F4D12C85
:10108000C12CE52EE694E694E694EC0CFD2CF11CC4
:10109000EC9EC001ED9E900DFC9E900D112403303E
:1010A00011F4880F991F289F7001299FF00C1124BB
:1010B000EE0DFF1D7D01EC0EFD1E1E141F040CF035
:1010C0006BC0A038B1050CF067C0CB01850F911D36
:1010D000181619060CF060C0603471050CF05CC085
:1010E000309709F459C0362F3770CB0177FD07963A
:1010F00023E0959587952A95E1F7282F77FF04C07F
:10110000332311F02FEF280F662777276A1B7B0BFD
:10111000B7FD02C070E060E090E89A1B40E8E4167A
:10112000F1040CF4912F961BE22E022E000CFF0806
:10113000DE2CD0942F3F0CF0D12C41E0852F87700E
:1011400009F440E0B52EB694B694B6944B0DE40E77
:10115000F11C89E0E816F10414F048E0421BB42EBB
:10116000BD182D0D40E8240370011124AE0DBF1DE4
:10117000A60FB71F1D9D600D711D1124AF01460FF5
:10118000571FC32E032E000CDD08033009F4C7C01F
:1011900090F4023009F474C0DF91CF911F910F9148
:1011A000FF90EF90DF90CF90BF90AF909F908F9087
:1011B0007F906F9008950A3FA1F1B20E0B3F61F747
:1011C0002B1551F3BD016A517D4F10E000E0091766
:1011D00008F09FC0FA01E00FF11FE491F0E04F0129
:1011E0000C2C02C0880C991C0A94E2F727FD06C05B
:1011F000FB018081F82CF0948F218083332361F0F0
:10120000273054F47B01F0E8EF0EF11CA92CA094D8
:10121000F70180818A2180830F5F1F4F6F5F7F4FAF
:10122000D6CFB20E2B1509F4B7CFBD016A517D4F51
:1012300010E000E0091708F066C0FA01E00FF11FA6
:10124000E491F0E04F010C2C02C0880C991C0A9428
:10125000E2F727FD04C0FB018081882980833323C6
:1012600051F0273044F47B01F0E8EF0EF11CF70158
:101270008081892980830F5F1F4F6F5F7F4FDACF97
:101280006FEF70E0032E02C0660F771F0A94E2F73B
:1012900060957095972E8B2C820E281509F47CCFC3
:1012A0008D010A511D4FF12CE12CE91630F5FA01A0
:1012B000EE0DFF1DE491F0E03F010C2C02C0660C26
:1012C000771C0A94E2F727FD05C0F8018081862388
:1012D00086298083332359F027304CF45801F0E8F5
:1012E000AF0EB11CF5018081892187298083FFEF32
:1012F000EF1AFF0A0F5F1F4FD8CF2F5F4C0F5D1FF4
:10130000A058BF4FCACF2F5F4C0F5D1FA058BF4FD3
:1013100089CF2F5F4C0F5D1FA058BF4F51CFE92ED3
:10132000F12CFA01E60FF71FAA51BD4F60E870E0FB
:101330006E197F09CE19DF098E01000F111F41E0E0
:1013400050E07A01032E01C0EE0C0A94EAF7592FFF
:101350004B2D892E932ECF93DF93ED01EF96EF96D1
:101360002296A590C590992059F0AE9C5001CE9C34
:10137000600127302CF4F880D094FD20FB28F992EE
:1013800022233AF0FC90C094FC20FA28FD920C94A1
:10139000CA0911965A9529F74A9551F0582D239567
:1013A0001124E00FF11DA60FB11DC60FD11DD9CF1D
:1013B000DF91CF911124F0CE0F9302E020E00E9444
:1013C00021080F9108952F923F924F925F926F9252
:1013D0007F928F929F92AF92BF92CF92DF92EF92C5
:1013E000FF920F931F93CF93DF93CDB7DEB728976C
:1013F0000FB6F894DEBF0FBECDBF6F836A0119012F
:101400001C830B83FE82ED82811128C005E010E071
:1014100029E030E03A832983B6010D2C000C880BBB
:10142000990B0E9415304B015C015F8151111DC069
:10143000E4E5F7E090E080E018861F828C159D05BA
:101440000CF02BC1248135814F81588542175307F9
:1014500014F438872F8301963696F0CF04E010E01D
:1014600048E050E05A834983D7CF20E030E040E0A5
:101470005FE30E9474304B015C0120E030E0A90181
:101480000E944F3320E030E040E05FE387FD30C052
:10149000C501B4010E94E3310E94C13278876F8395
:1014A000A6018F819885481B590BE4E5F7E090E091
:1014B00080E0B12CA12C2F81388582179307ECF0A6
:1014C00086E0829FF001839FF00D1124EC5AF84FC3
:1014D00090E080E0D12CC12C84179507BCF42481C6
:1014E0003581C216D3060CF4690101963696F4CF05
:1014F000C501B4010E94E231CFCF24813581A2160B
:10150000B3060CF4590101963696D5CFB801110FE8
:10151000880B990B0E9415302B013C01B5016C0D15
:101520007D1D072E000C880B990B0E94153020E0C2
:1015300030E040EE5FE30E94E3316B017C0120E08C
:1015400030E040E05FE3C301B2010E9474309B01D0
:10155000AC01C701B6010E9474306B017C0120E030
:1015600030E0A9010E944F3320E030E040E05FE32B
:1015700087FD89C0C701B6010E94E3310E94C132D4
:1015800002E410E0061B170BF10111830083B50183
:10159000BB0C880B990B0E94153020E030E040EE28
:1015A0005FE30E94E331A30192010E9474304B017A
:1015B0005C0120E030E0A9010E944F3320E030E0E0
:1015C00040E05FE387FD64C0C501B4010E94E331E0
:1015D0000E94C132600F711FEB81FC8171836083B7
:1015E00029813A81B901330F880B990B0E9415307C
:1015F00020E030E040E05FE30E9474306B017C014A
:101600004F815885BA01550F880B990B0E941530F0
:101610009B01AC01C701B6010E9474306B017C01D3
:1016200020E030E0A9010E944F3320E030E040E0AC
:101630005FE387FD85C0C701B6010E94E3310E94C8
:10164000C1322AE230E0C901861B970BED81FE8191
:101650009183808328960FB6F894DEBF0FBECDBF6E
:10166000DF91CF911F910F91FF90EF90DF90CF907E
:10167000BF90AF909F908F907F906F905F904F90B2
:101680003F902F900895C701B6010E94E23176CFB6
:10169000C501B4010E94E2319BCFB801110F880B44
:1016A000990B0E94153020E030E040E05FE30E949B
:1016B00074302B013C01EF81F885BF01FF0F880BCF
:1016C000990B0E9415309B01AC01C301B2010E942D
:1016D00074302B013C0120E030E0A9010E944F331F
:1016E00020E030E040E05FE387FD25C0C301B201A8
:1016F0000E94E3310E94C13222E430E0C901861B1E
:10170000970BF101918380838FEF9FEFEB81FC8139
:101710009183808329813A81B901330F880B990B1A
:101720000E94153020E030E040E05FE30E9474301A
:10173000A501940171CFC301B2010E94E231DACF59
:10174000C701B6010E94E2317ACFFC018091E50227
:10175000882311F13FB7F89482E08093E90020914B
:10176000F200822F90E01816190614F481E090E040
:10177000882339F0289844E64093E4024091F10030
:101780004083222339F02091F200211103C02BE67F
:101790002093E8003FBF08958FEF9FEF08952FB784
:1017A000F89483E08093E9009091E800892F80729B
:1017B00095FF04C09091F20080E4891B2FBF08952B
:1017C0008091DC0281110DC082E08093D80284E018
:1017D0008093D9021092DB021092DA0281E08093AA
:1017E000DC0288ED92E00895CF93DF931F92CDB78E
:1017F000DEB76983DC01ED91FC910280F381E02D7D
:1018000041E050E0BE016F5F7F4F09950F90DF917F
:10181000CF91089583E08093E9008091F2008823BE
:1018200019F08AE38093E80008950E94CF0B90E0BE
:101830000895CF93DF931F92CDB7DEB7FC01848567
:10184000958597FD08C02FEF3FEF358724870F90D0
:10185000DF91CF910895CE0101960E94A50B0197CB
:1018600019F4898190E0F3CF8FEF9FEFF0CF0F93C2
:101870001F93CF93DF931F92CDB7DEB78C01FC018E
:101880008485958597FF0BC0CE0101960E94A50B1C
:10189000019771F4898190E0F80195878487F801B8
:1018A000848595850F90DF91CF911F910F910895B9
:1018B0008FEF9FEFF1CFFC018485958597FD0BC0DD
:1018C0009FB7F89482E08093E9008091F2009FBF77
:1018D00090E0019608959FB7F89482E08093E90024
:1018E0008091F2009FBF90E008954091D202509104
:1018F000D3022091D0023091D10242175307B4F4A1
:101900009091E8009570E1F39091E80092FD19C084
:101910008093F1008091D2029091D30201968F734F
:101920009927892B19F48EEF8093E8008091D202D9
:101930009091D30201969093D3028093D20281E0DA
:10194000089580E00895DF92EF92FF920F931F9326
:10195000CF93DF93D82E8A01EB017B01E40EF51EB5
:10196000CE15DF0559F0D7FE12C0FE0184910E940A
:10197000750C21968111F4CF0FEF1FEFC801DF9195
:10198000CF911F910F91FF90EF90DF900895888184
:10199000EECF0F931F93CF93DF931F92CDB7DEB798
:1019A00082E0898342E450E064EE7EE080E80E94B9
:1019B000A30C0E94E00BDC0112960D911C91011505
:1019C000110589F0D801ED91FC910280F381E02DA1
:1019D000BE016F5F7F4FC801099597FD04C0F801F4
:1019E00000851185ECCF89810F90DF91CF911F91F8
:1019F0000F910895615030F02091F100FC01208397
:101A00000196F8CF289884E68093E40208953FB7C2
:101A1000F8948091CC029091CD02A091CE02B09129
:101A2000CF0226B5A89B05C02F3F19F00196A11D36
:101A3000B11D3FBFBA2FA92F982F8827BC01CD0118
:101A4000620F711D811D911D42E0660F771F881F77
:101A5000991F4A95D1F708958F929F92AF92BF92A6
:101A6000CF92DF92EF92FF926B017C010E94070DF3
:101A70004B015C01C114D104E104F104B9F00E94EE
:101A8000070D681979098A099B09683E7340810529
:101A9000910580F321E0C21AD108E108F10888EE2F
:101AA000880E83E0981EA11CB11CE4CFFF90EF903C
:101AB000DF90CF90BF90AF909F908F9008958F92BE
:101AC0009F92AF92BF92CF92DF92EF92FF920F93CD
:101AD0001F93CF93DF936C017B018A0180910C01EE
:101AE000882309F45CC08091E502882309F457C07B
:101AF0008091D70280FF05C08091E00082608093D2
:101B0000E000E801B12C8AEFA82E93E0892E2AE3A9
:101B1000922E209711F4BB20D9F10E94CF0B811196
:101B20000AC0AA94AA20D9F161E070E080E090E0B8
:101B30000E942C0DEECF8C171D0611F00CF08C2F8F
:101B40009FB7F8948092E9002091E80025FD02C03B
:101B50009FBFDFCF282F30E0C21BD30BF70181508E
:101B600020F041914093F100FACFE20EF31EBB202A
:101B700021F09092E800B12CEBCF8091E80085FD38
:101B8000E7CF9092E800BB24B394209709F3F3CFFA
:101B90005D9884E68093D602101611063CF081E031
:101BA00090E0F6019383828310E000E0C801DF91AA
:101BB000CF911F910F91FF90EF90DF90CF90BF904A
:101BC000AF909F908F9008950895DB0114964D91EA
:101BD0005C9115976D917C91DC01ED91FC910280F7
:101BE000F381E02D09942F923F924F925F926F9272
:101BF0007F928F929F92AF92BF92CF92DF92EF929D
:101C0000FF920F931F93CF93DF9300D000D000D0AB
:101C1000CDB7DEB7782E662E5A0128E0422E512C21
:101C2000811103C099E0492E512CCE0101967C010F
:101C30008E010D5F1F4F9E012B5F3F4FA501662D4B
:101C4000872D0E94E309B5010B2C000C880B990B22
:101C50000E94153020E030E040E05FE30E947430E5
:101C60006B017C0120E030E0A9010E944F3320E0AD
:101C700030E040E05FE387FD24C0C701B6010E9469
:101C8000E3310E94C1328B0184E5C82E87E0D82E53
:101C9000049D1001059D300C149D300C1124F12C75
:101CA000E12C912C812C8A149B04B4F589819A81B2
:101CB000662019F0801691064CF42D818E0D9F1D23
:101CC0000BC0C701B6010E94E231DBCF2B81A70117
:101CD00042195309840F951F7720A1F0209389079B
:101CE0002093880780938A07B60184E897E00E94D2
:101CF000E50D9FEF891A990A86E0C80ED11CE40C05
:101D0000F51CD1CF209393072093920780939407DB
:101D1000B6018EE897E0EBCF26960FB6F894DEBFBB
:101D20000FBECDBFDF91CF911F910F91FF90EF902C
:101D3000DF90CF90BF90AF909F908F907F906F90EB
:101D40005F904F903F902F900895EF92FF920F93E6
:101D50001F93CF93DF938C017B01D0E0C0E0F701AC
:101D6000EC0FFD1F6491662361F0D801ED91FC91A9
:101D70000190F081E02DC8010995892B11F0219681
:101D8000EECFCE01DF91CF911F910F91FF90EF9099
:101D90000895AF92BF92CF92DF92EF92FF920F938E
:101DA0001F93CF93DF936C017B018B01040F151FF1
:101DB000EB015E01AE18BF08C017D10759F0699159
:101DC000D601ED91FC910190F081E02DC6010995BD
:101DD000892B79F7C501DF91CF911F910F91FF906A
:101DE000EF90DF90CF90BF90AF9008952D9A089517
:101DF000BC0190E080E00C942C0D8FB18095807F29
:101E0000669B88601C9B8460089581EC80937C00B5
:101E100085B1806F85B984B1877E84B984B1876EBE
:101E200084B95E9A5F988AB1806D8AB9769A6E9805
:101E300081B3806F81BB899880B38D7080BB80E552
:101E40008CBD81E08DBD85E090E00E94F80E5F9A28
:101E500085E090E00E94F80E5E985C98ECE2F8E075
:101E600084918EBD00000DB407FEFDCF319688E051
:101E7000E933F807A9F75C9A81E8809364008091C0
:101E80006500816080936500089590915E029823BB
:101E900029F490915F02982381E009F480E008958D
:101EA000CF93C82F0E94FD0E982F9C2381E09C1396
:101EB00080E0CF91089580E00C94DB078038910595
:101EC000B8F460347105A0F420E191E061FD94E084
:101ED00060FD990F62FD9295687F269FD0011124C5
:101EE000A80FAA51BD4F8C9140FF03C0892B8C9342
:101EF000089590958923FBCF2F923F924F925F9246
:101F00006F927F928F929F92AF92BF92CF92DF9209
:101F1000EF92FF920F931F93CF93DF937C016B019E
:101F200088248394912CD0E0C0E005E010E096EF87
:101F3000692E77247A942CEFA22EBB24BA94842F96
:101F40008470582E842F8270482E842F8870382EEB
:101F50004170242E219682E0880E911CA80CB91C99
:101F6000552091F041E0B8016C0D7D1DC7018C0F2B
:101F70009D1F0E945E0F41E0B6016C0F7D1FC801DE
:101F80008E0D9F1D0E945E0F442091F041E0B6012E
:101F9000601B710BC7018C0F9D1F0E945E0F41E0FB
:101FA000B6016C1B7D0BC8018E0D9F1D0E945E0F3C
:101FB000332091F041E0B6016C0F7D1FC701801BFB
:101FC000910B0E945E0F41E0B8016C0D7D1DC701B1
:101FD0008C1B9D0B0E945E0F222091F041E0B60108
:101FE0006C1B7D0BC701801B910B0E945E0F41E0B3
:101FF000B601601B710BC7018C1B9D0B0E945E0F0D
:10200000C017D10754F4B7FCA5CF0150110982E0E5
:10201000680E711CA60CB71C9DCFDF91CF911F914C
:102020000F91FF90EF90DF90CF90BF90AF909F9077
:102030008F907F906F905F904F903F902F9008957A
:102040002F923F924F925F926F927F928F929F92C8
:10205000AF92BF92CF92DF92EF92FF920F931F93B6
:10206000CF93DF93EC0141E06FE370E00E945E0FDD
:1020700041E065E370E0CE010E945E0F41E06AE35B
:1020800070E0CE0105960E945E0F41E06AE370E0C9
:10209000CE0105970E945E0F22242394312CF12C4F
:1020A000E12C05E010E036EF432E55245A944CEF16
:1020B000C42EDD24DA948FEFE81AF80A82E0280EA5
:1020C000311CC20CD31C47018C0E9D1E41E05801EF
:1020D0008AE3A80EB11CB501C4010E945E0F3E0147
:1020E0006E187F0841E0B501C3010E945E0F41E018
:1020F0008AE3A82EB12CA01AB10AB501C4010E942E
:102100005E0F41E0B501C3010E945E0F47018AE303
:10211000880E911C41E0B4015E01A00EB11EC50104
:102120000E945E0F41E0B4013E01601A710AC301D2
:102130000E945E0F9AE3892E912C8E189F0841E031
:10214000B401C5010E945E0F41E0B401C3010E94C9
:102150005E0FE016F1069CF0DF91CF911F910F9179
:10216000FF90EF90DF90CF90BF90AF909F908F90B7
:102170007F906F905F904F903F902F900895D7FC85
:102180009ACF0150110982E0480E511CC40CD51C95
:1021900092CF8F929F92AF92BF92CF92DF92EF92A7
:1021A000FF920F931F93CF93DF936D3089F0C09010
:1021B0005C02D0905D026A30D1F410925B02109202
:1021C0005A0288E0C80ED11CD0925D02C0925C0217
:1021D00081E090E0DF91CF911F910F91FF90EF9000
:1021E000DF90CF90BF90AF909F908F900895009117
:1021F0005A0210915B02E5E06E9FE0011124C45D7C
:10220000DC4F4801F12CF5E0E12CFF1629F0CE015E
:102210000196FE01E490EC01B12CA12C4E2D4170F1
:10222000B6016A0D7B1DC4010E945E0FE694FFEFAC
:10223000AF1ABF0A88E0A816B10481F7F394EFEF54
:102240008E1A9E0AF6E0FF12DECF0A5F1F4F109330
:102250005B0200935A02BCCFDF92EF92FF920F9382
:102260001F93CF93DF937C01D22E8B01040F111D9E
:10227000EB0177FF02C0D0E0C0E0C80101341105D6
:1022800014F080E490E0C817D9073CF44D2DBE014E
:10229000C7010E945E0F2196F0CFDF91CF911F9171
:1022A0000F91FF90EF90DF9008952F923F924F9201
:1022B0005F926F927F928F929F92AF92BF92CF92D6
:1022C000DF92EF92FF920F931F93CF93DF9300D093
:1022D00000D000D0CDB7DEB76C01762E542E490168
:1022E000602E98E0A92EB12C611103C089E0A82EC0
:1022F000B12CCE0101967C018E010D5F1F4F9E0116
:102300002B5F3F4FA401652D872D0E94E3090981B2
:102310001A81552011F1B401990C880B990B0E9478
:10232000153020E030E040E05FE30E9474301B0194
:102330002C0120E030E0A9010E944F3320E030E082
:1023400040E05FE387FD0CC0C201B1010E94E331B0
:102350000E94C132C616D70644F48D809E8009C003
:10236000C201B1010E94E231F3CF8B809C80C61A7A
:10237000D70ACA9CB001CB9C700DDA9C700D112459
:10238000060F171FC40104976620B1F061E070E0EA
:10239000711002C062E070E0060F171F6C01C601E9
:1023A0002FEFC21AD20AC814D90491F020E045E0F8
:1023B000B8010E942C11F3CF61E070E0711002C0EF
:1023C00062E070E0600F711F49E55FE00E94DC0988
:1023D00026960FB6F894DEBF0FBECDBFDF91CF912A
:1023E0001F910F91FF90EF90DF90CF90BF90AF9033
:1023F0009F908F907F906F905F904F903F902F9025
:1024000008950F93CF93DF93EC019E816A3059F4C6
:102410008D818C836985960F9E8381E090E0DF91AA
:10242000CF910F910895262F61E0690F2A3398F418
:10243000203378F5273249F140F4213261F1988553
:102440009C5F8C81890F8C83E8CF2C3231F12E3246
:10245000B1F72FE309C0213490F32B35C0F08FE999
:10246000820F27548A3158F7062E000C770B8C8187
:10247000082E000C990B3F810AEF313009F00BEF69
:1024800042E252E00E942108DACF21E4EDCF21544C
:10249000EBCF2C5FE9CF2EE3E7CF20E4E5CF0F931E
:1024A000CF93DF93EC019E816A3059F48D818C8348
:1024B0006985960F9E8381E090E0DF91CF910F9127
:1024C0000895262F61E0690F2A3398F4203378F5B8
:1024D000273249F140F4213261F198859D5F8C816A
:1024E000890F8C83E8CF2C3231F12E32B1F72FE3F4
:1024F00009C0213490F32B35C0F08FE9820F2754A7
:102500008A3158F7062E000C770B8C81082E000CB0
:10251000990B3F810AEF313009F00BEF4AE551E0AA
:102520000E942108DACF21E4EDCF2154EBCF2C5FBC
:10253000E9CF2EE3E7CF20E4E5CFE2EAF2E02AEBB1
:1025400032E090E080E04191519161917191840F6E
:10255000951F2E173F07B9F74091710250917202F3
:1025600065E0649F9001659F300D1124280F391F8D
:1025700080916F0290917002821B930B0895CF930C
:10258000C82F84E00E94450F811107C0CC2381F041
:1025900088E00E94450F882359F01092C60280916E
:1025A0008102909182029093C3028093C20281E0E3
:1025B000CF910895E4E8F7E08AE48583848387E394
:1025C000868369ED70E0CF010E94A50E8BE490E058
:1025D0000E94201087E690E00C942010CF92DF92AA
:1025E000EF92FF920F931F93CF93DF9346E770E034
:1025F00060E085E090E00E94EA0746E76FE370E064
:1026000085E090E00E94EA0721E046E365E070E0A3
:1026100090E080E00E942C1121E046E365E070E04C
:102620008FE790E00E942C1141E065E070E085E0CA
:1026300090E00E947C0F42E065E070E08AE790E065
:102640000E947C0F44E06AE370E08AE790E00E9419
:102650007C0F48E06AE370E085E090E00E947C0F28
:1026600080918302C6E3D7E0811122C00AE010E026
:10267000F12CE12C8AE0C82ED12C8091840290911B
:102680008502E816F90684F58FEFE81AF80AD09269
:102690005B02C0925A0210935D0200935C02BE017D
:1026A00088E997E00E94E50D065F1F4F2696E5CF6B
:1026B0001AE0F12CE12C0AE08091840290918502CD
:1026C000E816F9068CF40093930700939207109391
:1026D0009407BE018EE897E00E94E50D8FEFE81A9F
:1026E000F80A175F2696E8CFDF91CF911F910F91DF
:1026F000FF90EF90DF90CF900895BC01EEE8F7E0F7
:1027000096E0958394838CE08683CF010C94E50D4D
:1027100090E080E008958F929F92AF92BF92EF92E7
:10272000FF920F931F93CF93DF93CDB7DEB7A1979F
:102730000FB6F894DEBF0FBECDBF7C01FA01CB010E
:1027400019A2223008F42AE08E010F5D1F4F822E5D
:10275000912CB12CA12CBF01A50194010E94B13193
:10276000F901CA016A3074F5605DD8016E938D017C
:10277000232B242B252B79F790E080E0109789F00C
:10278000FD0101900020E9F73197AF014A1B5B0B77
:10279000D701ED91FC910280F381E02DB801C701D2
:1027A0000995A1960FB6F894DEBF0FBECDBFDF919D
:1027B000CF911F910F91FF90EF90BF90AF909F909E
:1027C0008F900895695CD1CFCF92DF92EF92FF9204
:1027D0000F931F93CF93DF9377FF21C06A017B0193
:1027E000EC01E881F9810190F081E02D6DE209951D
:1027F0008C0144275527BA014C195D096E097F09E0
:102800002AE0CE010E948B13800F911FDF91CF91A0
:102810001F910F91FF90EF90DF90CF9008952AE0E5
:10282000DF91CF911F910F91FF90EF90DF90CF90AC
:102830000C948B13CF93DF93CFE1D0E020E04AE0FC
:1028400067E170E0CE010E942C112196CF36D105B0
:10285000A9F783E2809393078093920788E180939E
:10286000940740916B0250916C0260916D027091DF
:102870006E028EE897E0DF91CF910C94E413BC01D7
:10288000EEE8F7E09AE09583948388E18683CF01B0
:102890000E94E50D48E566E170E08EE190E00E945F
:1028A000EA0748E561E270E08EE190E00E94EA0705
:1028B00021E04CE066E170E08EE190E00E942C1196
:1028C00021E04CE066E170E085E790E00E942C1189
:1028D0000E941A1442ED50E068E170E08FE690E04B
:1028E0000C94DC09CF92DF92EF92FF920F931F932B
:1028F000CF93C82F8B0169017A016E5F7F4F4BEC3C
:1029000050E00E94DC09CA5FEEE8F7E0C583C483AB
:102910000683B701A601CF01CF911F910F91FF90C0
:10292000EF90DF90CF900C94E413CF93DF938091DE
:10293000C2029091C3024197029768F5C8E2D0E0C5
:1029400020E047E065E270E0CE010E942C11219664
:10295000CF37D105A9F7E0917F02F0918002EE0F09
:10296000FF1FEE0FFF1FE657FD4F2081318142818F
:10297000538160916B0270916C0280916D02909115
:102980006E020E94A1339B01AC0165E270E088E217
:1029900090E00E947214DF91CF910C941A14CF939F
:1029A000DF93EC0188819981009711F00E945334E4
:1029B000198218821D821C821B821A82DF91CF919C
:1029C0000895FC0180819181009711F00C9453349B
:1029D0000895CF93C82F8091C0029091C1020196B3
:1029E0009093C1028093C00210926A020E94452F08
:1029F00021EE3EE240E050E00E9448316058714CC8
:102A00008F4F9F4F60938A0270938B0280938C024A
:102A100090938D020E94452F29E53BE140E050E074
:102A20000E94483168577C4E8F4F9F4F60938E02B3
:102A300070938F0280939002909391020E94452F91
:102A400023E230E040E050E00E9448319B01AC01BD
:102A5000265F3F4F4F4F5F4FA4E6B0E00E946731C3
:102A600060939202709393028093940290939502E4
:102A70000E94452F2BE230E040E050E00E944831B8
:102A80009B01AC012F5D3F4F4F4F5F4FAAE0B0E07D
:102A90000E94673160939602709397028093980228
:102AA000909399020E94452F20E130E040E050E0F1
:102AB0000E9448319B01AC01295F3F4F4F4F5F4F50
:102AC000AAE0B0E00E94673160939A0270939B0283
:102AD00080939C0290939D020E94452F25E030E058
:102AE00040E050E00E9448319B01AC012F5F3F4F16
:102AF0004F4F5F4FAAE0B0E00E94673160939E02A3
:102B000070939F028093A0029093A102CC23C1F105
:102B100060917702709178028091790290917A02A7
:102B20000E9415302DEC3CEC4CE85FE30E947430C1
:102B30000E94F7320E94C13260937702709378024C
:102B40008093790290937A0260917302709174027B
:102B500080917502909176020E94153024E13EEA40
:102B600047E85FE30E9474300E94F7320E94C1324E
:102B7000609373027093740280937502909376024F
:102B80001092C602CF9108950C9432310F931F9387
:102B9000CF93DF938C01EB01FC0180819181009741
:102BA000E1F06881798161157105A9F04281538155
:102BB0002C813D814217530770F00E94A2358C8111
:102BC0009D81F801958384831D821C82DF91CF91C2
:102BD0001F910F9108950E94533488819981F801C3
:102BE000918380838A819B81938382838C819D8161
:102BF00095838483198218821B821A82E5CF0F93F2
:102C00001F93CF93DF93EC0188819981009759F04E
:102C10002A813B812617370730F081E0DF91CF9181
:102C20001F910F9108958B016F5F7F4F0E94DC34DD
:102C3000009759F0998388831B830A832C813D81F7
:102C4000232B59F7FC011082E8CF80E0E7CFEF9209
:102C5000FF920F931F93CF93DF93EC017B01CB0186
:102C60000E94A42F0097A9F00C811D81080F191F45
:102C7000B801CE010E94FF15882361F028813981B7
:102C80008C819D81B701820F931F0E949D2F1D8310
:102C90000C8381E0DF91CF911F910F91FF90EF9016
:102CA0000895EF92FF920F931F93CF93DF93FB0151
:102CB000E080F180E114F10441F480E0DF91CF91F4
:102CC0001F910F91FF90EF900895048115810115D8
:102CD0001105B1F0EC018C819D81080F191FB8011D
:102CE000CE010E94FF15882341F3288139818C8110
:102CF0009D81B701820F931F0E94A2351D830C8313
:102D000081E0DCCFEF92FF920F931F93CF93DF937D
:102D1000EC018B016115710551F0CB010E94A42FCC
:102D20007C01BC01CE010E94FF1581110BC0CE01B8
:102D30000E94CF14CE01DF91CF911F910F91FF9090
:102D4000EF900895FD82EC82B801888199810E94FC
:102D50009D2FF0CFFC011182108213821282158206
:102D600014820C948216CF93DF93EC0162307105CC
:102D700001F148F46115710581F061307105B1F020
:102D80006FE271E00CC064307105C9F0A8F06530E5
:102D90007105B1F760E371E002C06EE471E0CE014D
:102DA0000E94AA16CE01DF91CF91089566E471E0EA
:102DB000F6CF61E471E0F3CF6CE371E0F0CF66E34E
:102DC00071E0EDCFCF93DF93EC016230710501F13B
:102DD00048F46115710581F061307105B1F065EE5F
:102DE00070E00CC064307105C9F0A8F06530710561
:102DF000B1F766EE70E002C062E271E0CE010E94BF
:102E0000AA16CE01DF91CF91089565E171E0F6CF6A
:102E10006BE071E0F3CF6EEF70E0F0CF63EF70E046
:102E2000EDCFEF92FF920F931F93CF93DF93EC01BF
:102E30007B018A01BA010E94FF1581110BC0CE01EE
:102E40000E94CF14CE01DF91CF911F910F91FF907F
:102E5000EF9008951D830C83B701888199810E94AA
:102E6000A235F0CFFB0101900020E9F73197AF01C7
:102E7000461B570B0C9411170F931F93CF93DF939F
:102E8000CDB7DEB762970FB6F894DEBF0FBECDBFE9
:102E90008C01CB01F80111821082138212821582FB
:102EA00014824AE0BE016F5F7F4F0E94AD2FBE01CA
:102EB0006F5F7F4FC8010E94321762960FB6F89479
:102EC000DEBF0FBECDBFDF91CF911F910F9108954F
:102ED0000F931F93CF93DF93CDB7DEB7A2970FB6B3
:102EE000F894DEBF0FBECDBF8C01CB01BA01F80153
:102EF0001182108213821282158214822AE0AE019E
:102F00004F5F5F4F0E94B82FBE016F5F7F4FC801B8
:102F10000E943217A2960FB6F894DEBF0FBECDBF47
:102F2000DF91CF911F910F9108952F923F924F9271
:102F30005F926F927F928F929F92AF92BF92CF9249
:102F4000DF92EF92FF920F931F93CF93DF93CDB752
:102F5000DEB762970FB6F894DEBF0FBECDBF2C016F
:102F60009E012F5F3F4F490139011C01D12CC12C1B
:102F700010E000E0B12CA12CF1014191519161913F
:102F800071911F01CE010D960E946817E988FA8899
:102F9000CE010D960E94E114B601CE010D960E945D
:102FA000B31689899A89E80EF91EFFEFEF1AFF0A16
:102FB000F301E192F1923F01CE010D960E94E114DE
:102FC000F3E0CF16D1040CF03FC0AE14BF040CF4F4
:102FD00057012FEFC21AD20A36E0C316D10461F6A8
:102FE00084E5C82E87E0D82EF12CE12C150183E072
:102FF000E816F1040CF01801B701CE010D960E94FD
:10300000B316BE01635F7F4FC6010E94C615CE0195
:103010000D960E94E11468E571E0C6010E94271632
:10302000712C612CF401808191819101281B390B55
:103030006216730674F466E571E0C6010E942716F5
:103040003FEF631A730AEECF0E151F0514F68701C2
:10305000C0CFF20141915191619171912F01CE0147
:103060000D960E946817BE01635F7F4FC6010E94E4
:103070005116CE010D960E94E114FFEFEF1AFF0AE0
:1030800026E0C20ED11C32E0830E911C86E0E816C9
:10309000F10409F0ABCFF092BF02E092BE0281E0F2
:1030A0008093BC020A0D1B1D073111050CF480E052
:1030B0008093BD0262960FB6F894DEBF0FBECDBFFF
:1030C000DF91CF911F910F91FF90EF90DF90CF9004
:1030D000BF90AF909F908F907F906F905F904F9038
:1030E0003F902F900895EF92FF920F931F93CF93ED
:1030F000DF9300D000D000D0CDB7DEB78091C20200
:103100009091C302099709F05EC00E949D128C0144
:10311000BC01CE0101960E943C17ED80FE80CE01DD
:1031200001960E94E11481E08093890780938807CB
:1031300010928A0764EC70E084E897E00E94A50E84
:103140004091710250917202052E000C660B770BB4
:1031500084E897E00E94E41387E190E08E199F09CC
:10316000880F991F880F991F80938907809388077C
:1031700010928A076AEB70E084E897E00E94A50E3F
:10318000A801110F660B770B84E897E00E94E41307
:1031900010E000E021E041E068E070E0C8010E943A
:1031A0002C110F5F1F4F00381105A1F726960FB69F
:1031B000F894DEBF0FBECDBFDF91CF911F910F916D
:1031C000FF90EF90089540917B0250917C026091B6
:1031D0007D0270917E02CE0101960E946817ED80FB
:1031E000FE80CE0101960E94E11400E210E00E196B
:1031F0001F09000F111F000F111F8091C202909133
:10320000C3029C01255031092230310508F052C01B
:1032100021E0209389072093880710928A0760EBAA
:1032200070E0059711F465EB70E084E897E00E9488
:10323000A50E4BEC50E061E070E083E190E00E946D
:10324000DC0989E1809389078093880710928A07B7
:103250008091C2029091C302059719F540917702BF
:10326000509178026091790270917A0284E897E037
:103270000E94E4134BEC50E061E070E0C801069757
:103280000E94DC09009389070093880710928A073F
:1032900040917B0250917C0260917D0270917E0290
:1032A00073CF4091730250917402609175027091D6
:1032B0007602DCCF81E080938907809388071092A3
:1032C0008A076CEA70E084E897E00E94A50E8EE021
:1032D000809389078093880710928A074091C002E3
:1032E0005091C102052E000C660B770BBFCF1F92C9
:1032F0000F920FB60F9211248F939F938091E1004C
:103300009091E100937F9093E10083FF0FC01092B2
:10331000E90091E09093EB001092EC0092E390931F
:10332000ED001092E50298E09093F00082FF22C039
:1033300093E09093E9009091F200992319F09AE3B9
:103340009093E8009091D602992341F09091D60293
:1033500091509093D602911101C05D9A9091E40230
:10336000992341F09091E40291509093E4029111DD
:1033700001C0289A84FF18C08091E2008E7E81608F
:103380008093E2008091E1008F7E8093E100809144
:10339000D7028E7E80618093D7029F918F910F908C
:1033A0000FBE0F901F90189580FFF7CF8091E2001D
:1033B0008E7E80618093E2008091E1008E7E80931A
:1033C000E1008091D7028E7E8160E5CF1F920F923F
:1033D0000FB60F921124CF92DF92EF92FF920F93CC
:1033E0001F932F933F934F935F936F937F938F938D
:1033F0009F93AF93BF93EF93FF93CF93DF93CDB79B
:10340000DEB76C97DEBFCDBF1092E9008091E80077
:1034100083FF25C068E0CE0145960E94FA0C82EF3A
:103420008093E8008D8987FF39C09091E80090FF74
:10343000FCCF982F907609F034C19E894F89588D22
:103440002F89F88C911131C0803861F58091D502B7
:103450008093F1001092F1008EEF8093E8006C965B
:103460000FB6F894DEBF0FBECDBFDF91CF91FF91B5
:10347000EF91BF91AF919F918F917F916F915F91EC
:103480004F913F912F911F910F91FF90EF90DF90FF
:10349000CF900F900FBE0F901F9018959EEF9093B6
:1034A000E800C7CF1092F100D5CF913059F48111C7
:1034B000D3CF4130510581F68091D5028D7F809325
:1034C000D502CACF933049F48111C6CF413051059E
:1034D00019F68091D5028260F2CF953041F4809147
:1034E000E80080FFFCCF20682093E300B5CF963042
:1034F00009F0A9C00B8D1C8D22E01092E9001092FA
:10350000D3021092D202F2122EC01092D102109267
:10351000D0020E94C90C1F8299E09983FA8291E03F
:103520009E8390EA98879AEF99872091D2023091F2
:10353000D302275F3F4F3C832B838D831092E9009A
:103540001092D3021092D2021093D1020093D002B3
:1035500049E050E0BE016F5F7F4F80E00E94A30C06
:103560000E94C90C79CF1093D1020093D0020E941F
:10357000E00BDC0112960D911C910115110509F467
:1035800051C1D801ED91FC910480F581E02DBE017F
:103590006B5E7F4FC8010995009709F03EC1F801A5
:1035A00000851185EACFF3E0FF120EC08F898823D2
:1035B00009F440C0823061F440E860E188E49FE0B3
:1035C0000E94621C811148CF81E28093EB0047CFBB
:1035D000813029F440E86BE08CE39FE0F1CF833049
:1035E00099F70E94E00BDC011296ED90FC908E01A1
:1035F0000F5F1F4F6801E114F10479F0D701ED91DD
:10360000FC910680F781E02DB801C7010995080FEC
:10361000111DF701E084F184EECFD8011C92F60170
:1036200001900020E9F73197BF016C197D0940E056
:10363000C601C6CF66E27FE0FB01449150E080E81E
:103640000E94A30C09CF973009F4BECF983021F423
:1036500081E08093F10000CF993009F0FDCE8370B6
:1036600009F0B2CFE8E1F1E081E031E096E32191A9
:10367000222371F08093E9003093EB00DF01119772
:103680002C912093EC009093ED008F5F873079F7B9
:103690008EE78093EA001092EA008F898093E5021A
:1036A000DBCE8B8D9C8D1092E9001092D30210928C
:1036B000D2029093D1028093D002898D811192C061
:1036C0008E899D89913A49F4813209F07DCF47E096
:1036D00050E065E071E080E0B3CF913209F074CF43
:1036E000833269F48F89988DB0E0A0E08093010166
:1036F00090930201A0930301B0930401ADCE8032F8
:1037000069F48091E80082FFFCCF67E085E091E0FA
:103710000E94FA0C8BEF8093E8009ECE823209F073
:103720009BCE8F8980930C01EEEFFFE785919491FA
:103730008B3F9C4D51F1E0E0F8E0809105019091C4
:103740000601A0910701B0910801803B9440A105BA
:10375000B105F1F480910C0180FD1AC0EE3F8AE0C2
:10376000F80789F587E797E7918380838091600068
:103770008093D40288E19BE00FB6F894A8958093DB
:1037800060000FBE9093600067CEEEEFFAE0D5CFF9
:10379000808191818737974709F05ECEA895809107
:1037A00060008861809360008091D4028093600003
:1037B000EE3F2AE0F20789F08091FE0A9091FF0A1D
:1037C0009183808349CE808191818737980751F218
:1037D0009093FF0A8093FE0AC5CF1092FF0A1092C1
:1037E000FE0A3ACE0E94E00BDC0112960D911C916C
:1037F0000115110509F4E8CED801ED91FC91019075
:10380000F081E02DBE016B5E7F4FC80109958111EB
:1038100023CEF80100851185EBCF181619060CF49C
:103820001BCED2CEF1E0FF12BECE6AE27FE004CF23
:103830001F920F920FB60F9211242F933F938F93E5
:103840009F93AF93BF938091C8029091C902A091BA
:10385000CA02B091CB023091C70223E0230F2D376B
:1038600058F50196A11DB11D2093C7028093C8028F
:103870009093C902A093CA02B093CB028091CC026C
:103880009091CD02A091CE02B091CF020196A11DE0
:10389000B11D8093CC029093CD02A093CE02B09341
:1038A000CF02BF91AF919F918F913F912F910F9038
:1038B0000FBE0F901F90189526E8230F0296A11DAA
:1038C000B11DD2CFEF92FF920F931F93CF93DF934F
:1038D000F82E192FE62E042F81E0860F880F0E9404
:1038E000750C83E00E94750CCF2DD12FEC0EFD2EB0
:1038F000F11CCE15DF05B9F007FF13C0FE0184915E
:103900000E94750C182F80E00E94750C812321966F
:103910008111EFCFDF91CF911F910F91FF90EF9029
:1039200008958881EDCF81E0F5CFCF93DF9310929A
:10393000E9061092E80688EE93E0A0E0B0E08093FC
:10394000EA069093EB06A093EC06B093ED0682E2B4
:1039500091E09093E7068093E6068FEF9FEF9093B8
:10396000F3068093F20610929B0710929A078CE45C
:1039700091E0909399078093980710929107109285
:10398000900780E491E090938F0780938E0798E0F2
:103990009093970781E08093960710929307109277
:1039A00094071092920780939507109287071092C0
:1039B000860724E331E030938507209384079093B2
:1039C0008D0780938C071092890710928A071092B6
:1039D000880780938B07C4E5D7E0198218821B8281
:1039E0001A821D821C8250E040E06EEE71E0CE0132
:1039F0000E941117269687E0C438D80771F7C6E3EE
:103A0000D7E0198218821B821A821D821C8250E024
:103A100040E06EEE71E0CE010E941117269687E01D
:103A2000C435D80771F7DF91CF910895CF93DF9315
:103A3000CDB7DEB760970FB6F894DEBF0FBECDBF2F
:103A4000789484B5826084BD84B5816084BD85B579
:103A5000826085BD85B5816085BD80916E00816085
:103A600080936E001092810080918100826080932B
:103A7000810080918100816080938100809180002D
:103A8000816080938000809191008260809391009A
:103A9000809191008160809391008091900081607D
:103AA000809390008091C10084608093C1008091D8
:103AB000C10082608093C1008091C10081608093C9
:103AC000C1008091C30081608093C3008091C000D9
:103AD00082608093C0008091C20081608093C200A8
:103AE00080917A00846080937A0080917A0082606D
:103AF00080937A0080917A00816080937A0080912F
:103B00007A00806880937A001092E5021092D502C4
:103B10001092D7028091D70081608093D70080EA0D
:103B20008093D80089B5806189BD89B5826089BDDF
:103B300009B400FEFDCF61E070E080E090E00E94FB
:103B40002C0D8091D8008F7C80618093D80080916B
:103B5000E000807F8093E0008091E1008E7E809382
:103B6000E1008DE08093E200559A209A0E94050FB3
:103B700082E480930001809164008E7F80936400D2
:103B800080917A00806480937A0080917A0086FD2B
:103B9000FCCF00917800109179000E94070DAB01D5
:103BA000BC01C801B0E0A0E0DC01992788276C01C6
:103BB0007D01C40ED51EE61EF71EC701B601209179
:103BC00064002160209364006115710581059105F1
:103BD00011F00E94942F1092C3021092C202109210
:103BE000C6020E94050F0E945B0F80E80E94500FE2
:103BF0008823A9F05C9885EA8EBD00000DB407FE0D
:103C0000FDCF5C9A2E982F982D9880916400806249
:103C10008093640081E083BF889513BEFCCF84E06D
:103C20000E94500F882309F448C02D9884E80E9410
:103C3000500F8823E1F00E94F60E88EC90E00E947D
:103C4000F80E2F9882E090E00E9432318F3F29F0E9
:103C50006FEF82E090E00E943A3184EF91E00E94A1
:103C6000F80E2F9A84E80E94500F8111FBCF84E157
:103C70000E94500F8823E1F00E94F60E88EC90E03D
:103C80000E94F80E2E9882E090E00E943231882344
:103C900029F060E082E090E00E943A3184EF91E008
:103CA0000E94F80E2E9A84E10E94500F8111FBCFE2
:103CB00088EC90E00E94F80EB2CF0E94F60E82E0EF
:103CC00090E00E94C415882309F441C03E9A3F9AAF
:103CD00081E090E00E94C41581FF13C0082F04709A
:103CE000302E82FD2E9801EF1FEFB8E0AB2EB12CE5
:103CF00080E40E94500F882369F12E9A2F9A0E9427
:103D0000F60E82E390E00E94F80E0E94FD0E8111F3
:103D1000F8CFE2E04E2E512C612C712C8FB7F89425
:103D20004091C8025091C9026091CA027091CB02C1
:103D30008FBF80915802882309F4D0C01092580296
:103D400080E090E0892B51F30E940000E7CF3E987D
:103D50003F98BECF332029F00430110511F42E9A7C
:103D60002F9881E00E94DB07980117FF04C02227EB
:103D70003327201B310B27703327C80117FD079607
:103D8000A3E095958795AA95E1F717FF05C00197E0
:103D9000A501421B530B9A01BC017695762F66272D
:103DA000779567956A517D4FF12CE12C2501421AD8
:103DB000530A8E3F5FEF950709F43EC0DB0150E0E8
:103DC00040E0F701E75CF74F4F013B01F0E86F0E71
:103DD000711C8F3F980781F0F401E40FF51FE49107
:103DE000022E01C0EE0F0A94EAF75496FC91549704
:103DF000EF2B5496EC93549721153105B9F0F4014B
:103E0000E40FF51F24906301C40ED51EE22DF0E0EF
:103E1000042C02C0F595E7950A94E2F7FE87ED873A
:103E2000F6012488FD852F2AF601248A4F5F5F4F13
:103E300011964835510569F60196F8E5EF0EF11C2B
:103E400060587F4F40EBE416F10409F0B2CF0E94B6
:103E50005B0F8FE090E00E94F80E0F5F1F4F09315B
:103E6000110509F045CF332011F02F9A2D9880E9E4
:103E700091E00E94F80E0E94F60E81E090E00E9410
:103E8000C41580FF3ECF8AE090E00E94C4159FEFEA
:103E9000980F9E3F08F035CF22E330E030935B026D
:103EA00020935A0228E330E030935D0220935C02B5
:103EB0000BE010E0682F88E997E00E94C910C80164
:103EC0000E94C4150F5F1F4F0131110599F70E9421
:103ED0005B0F88EE93E00E94F80E13CF8091590299
:103EE000942F981B892F90910001891748F48F5FB8
:103EF000891708F025CF81E083BF889513BE20CFB6
:103F000081E080935802409359028091560290912B
:103F100057020196909357028093560280915F0258
:103F200080935E020E94FD0E80935F028091C60224
:103F30008111F5C02091C2023091C302E6EEF2E099
:103F400081118FEF00248193819381938193039456
:103F5000D1F710925D0210925C0210925B021092F7
:103F60005A021092C5021092C4022130310561F448
:103F70008091C0029091C1024F9734F087E190E0A8
:103F80009093C3028093C2028091C2029091C302B7
:103F90008831910508F0AEC4FC01EF52F04E0C944C
:103FA000B133E91F2D20FC20D720D7207821A12173
:103FB000BA211F22B820AA22AA22AA22AA22B62205
:103FC000E2227F2201230123A423A423A423A423E8
:103FD00011244AE65EE070E060E090E080E00E943C
:103FE000DC094AE65EE070E060E082E690E00E9474
:103FF000DC098AE290E090935B0280935A028FE0A2
:1040000090E090935D0280935C0261E67EE088E937
:1040100097E00E94A50E81E7809389078093880727
:104020008AE380938A076CE57EE084E897E00E944B
:10403000A50E6AE47EE084E597E00E94821681E0A6
:1040400090E09093BF028093BE021092BD02109246
:10405000BC0241E050E060E04DC00E9473186091E6
:10406000BA027091BB02CE0101960E94E216CE0107
:1040700001960E947D13CE0101960E94E11460E436
:104080007EE084E597E00E94821665E37EE08AE5A3
:1040900097E00E9482166AE27EE080E697E00E9446
:1040A000821666E27EE086E697E00E9482168091A4
:1040B000BA029091BB02892B09F057C06BE17EE0F8
:1040C0008CE697E00E94821666E17EE082E797E048
:1040D0000E94821686E090E09093BF028093BE0219
:1040E0001092BD0281E08093BC024091BE025091CB
:1040F000BF0261E080E00E94F30D2091BE0230918A
:10410000BF0200E04091BC026091BD028091C402F8
:104110009091C5020E94551181E08093C602C09023
:10412000C202D090C302B8E1CB16D10408F07CC41F
:10413000F601E356FF4D0C94B1339724972497244E
:104140009724972497249724732BE72AE72AE72AB2
:10415000EB2AEB2AEB2AE72AE72AEB2A692C692CBF
:10416000692C692C692C692CE72A84E090E0B4CF93
:104170000E9473186BE07EE0CE0101960E94AA16A1
:10418000CE0101960E947D13CE0101960E94E1149A
:1041900082EA92E00E9495174091BE025091BF02C0
:1041A0006091BC028091BD020E94F30DB5CF0E94C8
:1041B00073188091C2029091C30261E07EE0039780
:1041C00011F066EF7DE0CE0101960E94AA16CE01A5
:1041D00001960E947D13CE0101960E94E1148AE8A7
:1041E00092E00E9495174091BE025091BF026091EB
:1041F000BC028091BD027FCF0E9473186CEE7DE0FF
:10420000CE0107960E94AA166091BA027091BB0275
:10421000CE0101960E94E216BE016F5F7F4FCE0174
:1042200007960E945116CE0101960E94E1141A824F
:1042300019821C821B821E821D826F817885611506
:10424000710531F04B855C85CE0101960E941117F6
:10425000CE0101960E947D13CE0101960E94E114C9
:1042600074E5E72E77E0F72E70E060E08B010F5FDA
:104270001F4F8091BA029091BB02681779070CF02A
:10428000B801CE0101960E94E216BE016F5F7F4F1A
:10429000C7010E94C615CE0101960E94E114A6E056
:1042A000EA0EF11CB8010530110501F71093BF02A9
:1042B0000093BE0281E08093BD028093BC0245E082
:1042C00050E061E00E94F30D2091BE023091BF02E8
:1042D00000E04091BC026091BD028091C4029091C7
:1042E000C5020E945511CE0107960E94E11414CF19
:1042F0000E94731861EE7DE0CE0101960E94AA161D
:10430000CE0101960E947D13CE0101960E94E11418
:1043100066ED7DE084E597E00E94821669EC7DE021
:104320008AE597E00E94821682E090E09093BF02B7
:104330008093BE021092BD021092BC0242E050E097
:104340008ACE0E94731864EC7DE0CE0101960E9433
:10435000AA16CE0101960E947D13CE0101960E94FD
:10436000E11466EB7DE084E597E00E94821667EA3F
:104370007DE0D6CF68E97DE086E397E00E94821673
:104380006DE87DE08CE397E00E94821660918802E0
:1043900070918902CE0101960E943C17BE016F5FA9
:1043A0007F4F8CE397E00E945116CE0101960E9448
:1043B000E11467E87DE08CE397E00E94271666E74A
:1043C0007DE082E497E00E94821668E67DE088E462
:1043D00097E00E9482166091860270918702CE015A
:1043E00001960E943C17BE016F5F7F4F88E497E003
:1043F0000E945116CE0101960E94E11484E090E0E3
:104400009093850280938402109283020E94EE12A0
:1044100082E4809389078093880787E380938A07E3
:104420006FE97CE084E897E00E94A50E83E490E0C9
:104430000E94201087E690E00E9420106DCE0E941E
:10444000452F6B017C016FE87CE086E397E00E94DA
:10445000821668E87CE08CE397E00E94821687E091
:1044600090E0909382028093810283E090E09093A9
:1044700085028093840210928302C701B601A301D2
:1044800092010E944831672B79F463E87CE08CE369
:1044900097E00E9427166AE77CE082E497E00E949A
:1044A00082160E94EE1238CE63E77CE08CE397E040
:1044B0000E94271669E67CE082E497E00E9482165B
:1044C0008091860290918702039790938702809350
:1044D0008602181619062CF369E57CE088E497E05B
:1044E0000E94821684E090E090938502809384027B
:1044F00087E190E09093820280938102D2CF66E5BB
:104500007DE086E397E00E94821668E47DE08CE31C
:1045100097E00E94821669E37DE082E497E00E94C2
:1045200082166DE27DE088E497E00E94821684E0C6
:1045300090E09093850280938402109283020E94FF
:10454000EE120E94DA1281E090E090938202809352
:104550008102E2CD0E94EE128091C2029091C302CC
:104560000A9709F4D9CD0E94DA12D6CD64E571E03C
:1045700086E397E00E94321767E671E08CE397E0EC
:104580000E9432176CE771E082E497E00E943217D4
:1045900060E971E088E497E00E94321762EA71E016
:1045A0008EE497E00E94321785E090E090938502B8
:1045B0008093840281E0809383020E94EE128FE058
:1045C00090E0C3CF6EEE71E086E397E00E94321771
:1045D00066EB71E08CE397E00E94321765EC71E0C6
:1045E00082E497E00E94321783E090E09093850286
:1045F00080938402109283020E94EE1287E190E081
:10460000A4CF66E27DE0419711F060E27DE086E3B1
:1046100097E00E94821660917F0270918002CE0125
:1046200001960E94B316BE016F5F7F4F86E397E04D
:104630000E945116CE0101960E94E1146CE27DE0C9
:104640008CE397E00E9482166BE27DE082E497E0C3
:104650000E9482168091C2029091C30261E17DE0C6
:10466000419711F06BE07DE088E497E00E948216AC
:1046700067E17DE08EE497E00E94821685E090E09D
:10468000909385028093840281E0809383020E944C
:10469000EE12E0917F02F0918002EE0FFF1FEE0F0D
:1046A000FF1FE657FD4F2081318142815381609188
:1046B0003A0770913B07E5E0E69FC001E79F900D48
:1046C00011246AE070E00F960E9472148091C20279
:1046D0009091C3024197E9F420917B0230917C02D2
:1046E00040917D0250917E026EE270E087E390E09F
:1046F0000E9472140E94951467E07DE0CE0101963D
:104700000E94AA16CE0101960E943F14CE01019686
:10471000ECCD87E380939307809392078EE280939A
:104720009407E0917F02F0918002EE0FFF1FEE0FE1
:10473000FF1FEE55FD4F40815181628173818EE8EC
:1047400097E00E94E413D6CF6CEF7CE083319105B3
:1047500059F06FEE7CE08431910531F061EE7CE040
:10476000459711F062ED7CE086E397E00E948216A7
:1047700066E07DE08CE397E00E94821665E07DE0D4
:1047800082E497E00E9482168091810290918202D9
:1047900061EC7CE0059711F069EB7CE088E497E040
:1047A0000E94821669EC7CE08EE497E00E948216FB
:1047B00085E090E0909385028093840281E080936D
:1047C00083020E94EE1280918102909182020597ED
:1047D000F9F420917702309178024091790250915A
:1047E0007A0265E270E082E390E00E947214209108
:1047F0007B0230917C0240917D0250917E026EE2FC
:1048000070E087E390E00E94721465EB7CE076CF65
:10481000209173023091740240917502509176029A
:10482000E0CF609173027091740280917502909153
:10483000760200917B0210917C0220917D023091E2
:104840007E02600F711F821F931F009177021091EB
:1048500078022091790230917A02601B710B820BF1
:10486000930B0E94153020E030E04CEF51E40E94A1
:104870004F320E945A330E94F7320E94C1326B01BC
:104880006EEE71E086E397E00E94321763ED71E00F
:104890008CE397E00E94321760EE71E082E497E0CB
:1048A0000E943217B6016536710514F064E670E0B7
:1048B000CE0101960E943C17BE016F5F7F4F82E4DC
:1048C00097E00E945116CE0101960E94E1146FEE0E
:1048D00071E088E497E00E9432171092830284E02E
:1048E00090E090938502809384021092820210924D
:1048F0008102D7CD85E090E090935B0280935A02CD
:1049000090935D0280935C026EEA7CE088E997E018
:104910000E94A50E4091C2025091C302052E000CC8
:10492000660B770B88E997E00E94E413F5CB80E8EB
:104930000E94450F81111AC080E10E94450F81112C
:1049400015C080E20E94450F811110C080E40E94D2
:10495000450F81110BC088E00E94450F811106C0F0
:1049600084E00E94450F882309F45EC0A090BE0237
:10497000B090BF023090BC02E090C402F090C5023B
:1049800001E09501432D6091BD02C7010E945511C0
:10499000B5010B2C000C880B990B0E94153020E000
:1049A00030E040E05FE30E9474306D877E878F8740
:1049B000988B20E030E0A9010E944F3320E030E0E6
:1049C00040E05FE387FD33C06D857E858F859889E4
:1049D0000E94E3310E94C1328B0188248394912C80
:1049E000E616F7061CF032E0832E912C80E10E943F
:1049F000450F882359F1EFEFEE1AFE0AEA14FB0483
:104A0000ECF4F092C502E092C4022091BE02309113
:104A1000BF0200E04091BC026091BD028091C402DF
:104A20009091C5020E9455110E945B0F89C96D8546
:104A30007E858F8598890E94E231CCCFF1E0AF1A54
:104A4000B108B092C502A092C402DFCF80E80E94F4
:104A5000450F882371F001E0E01AF108F092C502D9
:104A6000E092C402F7FED1CF1092C5021092C402A8
:104A7000CCCF80E40E94450F8823D9F03320A9F0E1
:104A80008A94892891F4E00EF11EF092C502E0921A
:104A9000C4028091C4029091C5028A159B050CF452
:104AA000B4CF41E0A41AB108CCCF3FEFE31AF30A28
:104AB000ECCF80E20E94450F8823B9F0332089F0C3
:104AC00052E08516910469F4E01AF10AF092C502E9
:104AD000E092C4028091C4029091C50297FF95CFE5
:104AE000C3CF81E0E81AF108F1CF88E00E94450FBA
:104AF000882309F459C51092C60293E0C916D1045F
:104B000009F4BFC308F05AC0B1E0CB16D10409F4D0
:104B100086C0E2E0CE16D10409F4B0C0EF2809F057
:104B200074CF81E090E09093C3028093C20220EDA5
:104B300037E040E050E020937B0230937C024093CA
:104B40007D0250937E0288E893E1A0E0B0E080937C
:104B5000770290937802A0937902B0937A02109230
:104B600073021092740210927502109276021092E3
:104B7000BB021092BA02109272021092710284E685
:104B800090E09093700280936F0282E390E09093A4
:104B9000870280938602E2EAF2E08AEB92E01192C9
:104BA0001192119211928E179F07C9F71092C102AC
:104BB0001092C00280E00E94E91427CFF5E0CF16E2
:104BC000D10409F47EC408F423C416E0C116D1044C
:104BD00009F0A4CF86E090E0909382028093810256
:104BE00010926B0210926C0210926D0210926E0283
:104BF000E114F10409F4C9C4EA94EF2809F005CFDF
:104C000086E190E09093C3028093C2028091730288
:104C100090917402A0917502B091760221C4D09255
:104C20008202C092810292E0E916F104F1F074F47C
:104C3000E114F104B9F084E090E0EA94EF2809F07F
:104C4000E4CE9093C3028093C202DFCEE4E0EE167E
:104C5000F10489F06CF086E090E005E0E016F104E4
:104C600081F3D3CE83E090E0ECCF89E090E0E9CF10
:104C700082E090E0E6CF85E090E0E3CF8091BA0259
:104C80009091BB02E816F9061CF01FEFE11AF10A39
:104C9000F092BB02E092BA0281E00E94E9140E9405
:104CA000452F24E130E040E050E00E9448319B0174
:104CB00041E050E0509382024093810210928302BF
:104CC000FB013197E131F10508F0D6C2E659F94D03
:104CD0000C94B1337B26A226C126F426F4261F2786
:104CE0001F274C27932793279327F527F527492834
:104CF0006A289928092963ED7BE086E397E00E9402
:104D0000821661EC7BE08CE397E00E94821668EBF0
:104D10007BE082E497E00E94821683E090E090932B
:104D200085028093840222E030E040E050E020934E
:104D30009E0230939F024093A0025093A1028AE00A
:104D400090E07FCF67EA7BE086E397E00E948216DF
:104D500067E97BE08CE397E00E94821682E090E0B6
:104D600090938502809384028AE790E0A0E0B0E00F
:104D70008093960290939702A0939802B093990221
:104D8000DECF66E87BE086E397E00E94821668E764
:104D90007BE08CE397E00E94821667E67BE082E48A
:104DA00097E00E9482166AE57BE088E497E00E9423
:104DB000821684E090E090938502809384020E94A2
:104DC000452F2EE734E040E050E00E9448316E5A13
:104DD0007C4F8F4F9F4F60938E0270938F02809312
:104DE000900290939102ABCF6AE47BE086E397E078
:104DF0000E9482166BE37BE08CE397E00E948216B0
:104E00006DE27BE082E497E00E94821663E27BE041
:104E100088E497E00E94821684E090E090938502F7
:104E2000809384020E94452F29EA31E640E050E059
:104E30000E944831605B794B8F4F9F4FCCCF64E12C
:104E40007BE086E397E00E94821663E07BE08CE3E0
:104E500097E00E94821660EF7AE082E497E00E9479
:104E6000821683E090E090938502809384020E94F2
:104E7000452F21E63AEE40E050E00E94483160586C
:104E8000774C8E4F9F4F60938A0270938B02809372
:104E90008C0290938D0253CF61EE7AE086E397E027
:104EA0000E94821665ED7AE08CE397E00E948216FC
:104EB00082E090E0909385028093840260917B026F
:104EC00070917C0280917D0290917E020E9415304B
:104ED00020E030E040E450E40E944F326B017C015E
:104EE00020E030E0A9010E944F3320E030E040E0B4
:104EF0005FE387FD13C0C701B6010E94E3310E9442
:104F0000C132660F771F881F991F60937B027093D1
:104F10007C0280937D0290937E0211CFC701B6017F
:104F20000E94E231ECCFE2EAF2E04AEB52E090E09C
:104F300080E0C190D190E190F1908C0D9D1D4E17B5
:104F40005F07B9F7C2970CF43FC382E090E02930C5
:104F5000310539F084E090E02A30310511F085E028
:104F600090E0909389028093880269EC7AE086E36E
:104F700097E00E94821664EC7AE08CE397E00E944E
:104F80008216609188027091890261507109CE0188
:104F900001960E943C17BE016F5F7F4F8CE397E044
:104FA0000E945116CE0101960E94E1146CEB7AE04A
:104FB0008CE397E00E94271660EB7AE082E497E0AA
:104FC0000E94821665EA7AE088E497E00E948216E1
:104FD00084E090E0909385028093840287E090E0E3
:104FE0009093820280938102AACE80917B0290915D
:104FF0007C02A0917D02B0917E02843F9140A10588
:10500000B1050CF4E1C20E949D1205970CF4DCC2BC
:105010000E94452F23E030E040E050E00E944831FC
:105020006B0166E97AE086E397E00E948216F2E07F
:10503000CF16D104C8F469E77AE0CD2811F069E60B
:105040007AE08CE397E00E94821669E87AE082E4D5
:1050500097E00E94821683E090E09093850280930F
:1050600084028BE090E0EDCD6BE57AE08CE397E095
:105070000E9482166DE47AE082E497E00E94821634
:1050800064E47AE088E497E00E94821684E090E08D
:10509000E4CF63E37AE086E397E00E94821663E25E
:1050A0007AE08CE397E00E94821661E17AE082E484
:1050B00097E00E94821660E07AE088E497E00E9420
:1050C000821684E090E090938502809384028DE0C4
:1050D00090E0B7CD80917B0290917C02A0917D02FF
:1050E000B0917E028C329140A105B1050CF46CC2E6
:1050F0006DEE79E086E397E00E9482166DED79E02F
:105100008CE397E00E9482166EEC79E082E497E0EF
:105110000E94821663EC79E088E497E00E94821690
:1051200084E090E090938502809384028CE090E08C
:1051300088CD0E949D1208970CF446C20E94452F0C
:1051400027E030E040E050E00E9448318B010F5FE3
:105150001F4F0E94452F26E030E040E050E00E94C3
:1051600048316B01FB01EE0FFF1FEE0FFF1FEE55E5
:10517000FD4FA801012E000C660B770B80819181F9
:10518000A281B381840F951FA61FB71F80839183CF
:10519000A283B38368EB79E086E397E00E948216EE
:1051A000B801CE0101960E943C17BE016F5F7F4F90
:1051B00086E397E00E945116CE0101960E94E11409
:1051C0006DEA79E08CE397E00E948216B601CE0189
:1051D00001960E94B316BE016F5F7F4F8CE397E08C
:1051E0000E945116CE0101960E94E1146DEF71E00C
:1051F00082E497E00E9432176FE072E088E497E063
:105200000E94321784E090E090938502809384029C
:1052100096CD6DE172E086E397E00E9432176CE272
:1052200072E08CE397E00E9432176EE372E082E452
:1052300097E00E9432176DE472E088E497E00E94E4
:10524000321784E090E090938502809384020E945C
:10525000452F27E232E040E050E00E94483166509E
:105260007F4F8F4F9F4F6093920270939302809372
:1052700094029093950263CD5093C3024093C2026F
:10528000C4CB0E949D128C01D0928202C0928102F6
:10529000F0928002E0927F0218161906F4F163E59D
:1052A0007CE086E397E00E94821662E57CE08CE376
:1052B00097E00E94821662E47CE082E497E00E941C
:1052C00082166CE37CE088E497E00E94821660918D
:1052D0007F0270918002CE0101960E94B316BE013A
:1052E0006F5F7F4F88E497E00E945116CE010196D0
:1052F0000E94E1146AE37CE088E497E00E942716AC
:1053000084E090E09093850280938402109283025F
:105310008091C2029091C30263CEF701EE0FFF1F8E
:10532000EE0FFF1FE657FD4FC080D180E280F38073
:1053300060917B0270917C0280917D0290917E024F
:105340006C157D058E059F0544F564E37CE086E3DE
:1053500097E00E94821663E37CE08CE397E00E9472
:10536000821662E27CE082E497E00E9482166091FD
:105370007F0270918002CE0101960E94B316BE0199
:105380006F5F7F4F88E497E00E94C615CE010196BB
:105390000E94E11460E27CE0AFCF21E130E0309385
:1053A000C3022093C20210926B0210926C02109200
:1053B0006D0210926E020E9415304B015C01C70114
:1053C000B6010E9415309B01AC01C501B4010E94D9
:1053D0004F320E94F7320E94C13260936002709394
:1053E00061028093620290936302012E000C220BF3
:1053F000330B06171707280739070CF006CB009365
:105400006002109361022093620230936302FDCA2E
:1054100084E090E09093820280938102F092800277
:10542000E0927F02F701EE0FFF1FEE0FFF1FEE5518
:10543000FD4F80819181A281B381181619061A0649
:105440001B06BCF422E130E03093C3022093C20279
:1054500010926B0210926C0210926D0210926E020A
:105460008093600290936102A0936202B093630202
:10547000CCCA6AE17CE086E397E00E94821669E18B
:105480007CE08CE397E00E94821666E07CE082E498
:1054900097E00E94821660917F0270918002CE0197
:1054A00001960E94B316BE016F5F7F4F88E497E0BC
:1054B0000E94C615CE0101960E94E11464E07CE0D2
:1054C0001BCFD0928202C092810210926B02109286
:1054D0006C0210926D0210926E02E114F10419F147
:1054E000EA94EF2809F091CA80916A028823D1F1E9
:1054F00068EF7BE086E397E00E94821669EE7BE02E
:105500008CE397E00E94821662EE7BE082E497E0F3
:105510000E94821683E090E090938502809384023B
:10552000109283020CCC83E190E09093C3028093AD
:10553000C20240917B0250917C0260917D02709189
:105540007E028091770290917802A0917902B091C9
:105550007A02481759076A077B070CF081CFDB01F5
:10556000CA017ECF84E190E09093C3028093C2028F
:1055700028E833E140E050E020936002309361027C
:10558000409362025093630240CA85E190E0909399
:10559000C3028093C20280917B0290917C02A09111
:1055A0007D02B0917E025CCF84E00E94450F88238B
:1055B00009F42BCA42E0C41AD10855E0C516D1043B
:1055C00008F023CA1092C60281E090E03ACB81E055
:1055D0000E94BF1229CA80E00E94BF12811124CA12
:1055E00088E00E94450F882309F41ECA1092C60263
:1055F0008091C2029091C3028C30910509F44EC093
:1056000060F50B9709F010CA8091710290917202B7
:105610000196909372028093710280917B02909127
:105620007C02A0917D02B0917E0280599140A10937
:10563000B10980937B0290937C02A0937D02B0938A
:105640007E0280916F029091700205979093700294
:1056500080936F0281E090E041C08D309105E1F1CF
:10566000409709F0E1C980917B0290917C02A09162
:105670007D02B0917E02885E9340A109B1098093BA
:105680007B0290937C02A0937D02B0937E0282E322
:1056900090E09093870280938602DCCF80916F0226
:1056A000909170020A969093700280936F0280919D
:1056B0007B0290917C02A0917D02B0917E02885C79
:1056C0009109A109B10980937B0290937C02A09378
:1056D0007D02B0937E02BECF8EE090E09093C30235
:1056E0008093C202A1C984E00E94450F882309F477
:1056F00040C01092C6020E94452FA30192010E9451
:105700004831672B682B692BB9F46CE979E086E3A3
:1057100097E00E94821661E979E08CE397E00E94AD
:10572000821682E090E0909385028093840210922A
:10573000830281E090E016C061E879E086E397E0BB
:105740000E9482166BE779E08CE397E00E94821654
:1057500082E090E09093850280938402109283020D
:1057600088E090E090938202809381028AE090E04A
:10577000B5CF88E00E94450F882309F455C91092DF
:10578000C6028091710290917202892BE9F46CE655
:1057900079E086E397E00E9482166DE579E08CE37C
:1057A00097E00E94821660E579E082E497E00E942B
:1057B000821683E090E09093850280938402109299
:1057C000830287E090E0CECF0E94452FA301920193
:1057D0000E944831672B682B692B49F46FE479E00C
:1057E00086E397E00E9482166FE379E0ADCF809167
:1057F0008802909189020197909389028093880290
:10580000181619064CF46EE379E086E397E00E94DF
:1058100082166EE279E098CF0E94452F23EE34E0A5
:1058200040E050E00E9448318B0102511D4F6CE175
:1058300079E086E397E00E9482166EE079E08CE3DF
:1058400097E00E948216B801CE0101960E943C1793
:10585000BE016F5F7F4F8CE397E00E945116CE012F
:1058600001960E94E1146CEF78E082E497E00E94D8
:10587000821669EE78E088E497E00E94821684E060
:1058800090E0909385028093840281E0809383026C
:10589000012E000C220B330B80917B0290917C0235
:1058A000A0917D02B0917E02800F911FA21FB31FB5
:1058B00080937B0290937C02A0937D02B0937E0242
:1058C000803B9440A105B1050CF433CF80E190E01A
:1058D00049CF80E00E94BF128111A6C888E00E94D3
:1058E000450F882309F439C18091C2029091C30207
:1058F0008331910509F4B7C068F48131910509F449
:1059000079C04297C1F11092C602809181029091B4
:105910008202E4CE8531910509F402C108F4CCC0BD
:10592000469789F740916B0250916C0260916D022D
:1059300070916E028091730290917402A091750231
:10594000B0917602841B950BA60BB70B8093730264
:1059500090937402A0937502B093760280917B02BB
:1059600090917C02A0917D02B0917E02840F951FE0
:10597000A61FB71F36C080917F02909180022091B0
:105980006B0230916C0240916D0250916E02880F53
:10599000991F880F991FFC01EE55FD4FC080D180E3
:1059A000E280F380C21AD30AE40AF50AC082D182E7
:1059B000E282F38286579D4FDC016D917D918D913E
:1059C0009C910E94A13300917B0210917C02209156
:1059D0007D0230917E02DC01CB01800F911FA21F5E
:1059E000B31F80937B0290937C02A0937D02B093BF
:1059F0007E0289CF80917F029091800220916B027C
:105A000030916C0240916D0250916E02880F991F87
:105A1000880F991FFC01EE55FD4FC080D180E280B8
:105A2000F380C20ED31EE41EF51EC082D182E28234
:105A3000F38286579D4FFC01608171818281938141
:105A40000E94A13300917B0210917C0220917D0283
:105A500030917E0268017901C61AD70AE80AF90A6C
:105A6000D701C601BECF40916B0250916C0260918C
:105A70006D0270916E028091770290917802A091F0
:105A80007902B0917A02841B950BA60BB70B809319
:105A9000770290937802A0937902B0937A02809172
:105AA0007B0290917C02A0917D02B0917E02841BCA
:105AB000950BA60BB70B95CF40916B0250916C02E2
:105AC00060916D0270916E028091770290917802E0
:105AD000A0917902B0917A02840F951FA61FB71F7B
:105AE0008093770290937802A0937902B0937A0220
:105AF00080917B0290917C02A0917D02B0917E0208
:105B0000840F951FA61FB71F80937B0290937C0282
:105B1000A0937D02B0937E0281E080936A02F3CE6F
:105B200040916B0250916C0260916D0270916E0217
:105B30008091730290917402A0917502B0917602E7
:105B4000840F951FA61FB71F809373029093740252
:105B5000A0937502B0937602A2CF8FB7F894C0904D
:105B6000C802D090C902E090CA02F090CB028FBF69
:105B70008091C2029091C302419701E010E0029728
:105B800010F00AE010E08091660290916702A09107
:105B90006802B0916902B701A601481B590B6A0B54
:105BA0007B0B8091640290916502823091050CF02C
:105BB000F5C0453F51406105710510F40C94142562
:105BC0000196909365028093640280E80E94500FD2
:105BD0008823C1F1C0926602D0926702E092680207
:105BE000F09269028091600290916102A09162023C
:105BF000B0916302012E000C220B330B40916B021B
:105C000050916C0260916D0270916E026C017D0189
:105C1000C01AD10AE20AF30AC416D506E606F70648
:105C20000CF447C0040F151F261F371F00936B028B
:105C300010936C0220936D0230936E020E949514B3
:105C40000C94142580E40E94500F882309F443C06B
:105C5000C0926602D0926702E0926802F0926902F6
:105C60004091600250916102609162027091630202
:105C70002AE0209FC001219F900D1124092E000CC5
:105C8000AA0BBB0B00916B0210916C0220916D026C
:105C900030916E026A017B01C81AD90AEA0AFB0A2E
:105CA000C016D106E206F3066CF0800F911FA21F0A
:105CB000B31F80936B0290936C02A0936D02B0931C
:105CC0006E02BCCF40936B0250936C0260936D02E6
:105CD00070936E02B3CF80E10E94500F882339F198
:105CE000C0926602D0926702E0926802F092690266
:105CF000012E000C220B330B80916B0290916C02F1
:105D0000A0916D02B0916E0280179107A207B307B0
:105D10002CF0801B910BA20BB30BCBCF10926B021C
:105D200010926C0210926D0210926E0287CF80E288
:105D30000E94500F882321F1C0926602D092670220
:105D4000E0926802F09269028AE0809FA001819F40
:105D5000500D1124052E000C660B770B80916B0201
:105D600090916C02A0916D02B0916E02841795071C
:105D7000A607B7079CF2841B950BA60BB70B99CF10
:105D800010926602109267021092680210926902E5
:105D900010926502109264020C9414254536510548
:105DA0006105710508F011CF0C941425CF93DF9392
:105DB0008EE497E00E94E11488E497E00E94E114E9
:105DC00082E497E00E94E1148CE397E00E94E114E2
:105DD00086E397E00E94E114C4E8D7E02697CE015D
:105DE0000E94E11487E0C435D807C1F7DF91CF9155
:105DF00008958F929F92AF92BF92CF92DF92EF92CF
:105E0000FF92CF93DF93EC01688179818A819B8136
:105E1000611571058105910521F464E279ED8BE549
:105E200097E02DE133EF41E050E00E944831490115
:105E30005A019B01AC01A7EAB1E40E9467316B01F2
:105E40007C01ACEEB4EFA50194010E947531C60E41
:105E5000D71EE81EF91EF7FE06C081E0C81AD10859
:105E6000E10880E8F80AC882D982EA82FB82C70189
:105E7000B6019F77DF91CF91FF90EF90DF90CF90A9
:105E8000BF90AF909F908F9008958F929F92AF9206
:105E9000BF92CF92DF92EF92FF9260910D017091CD
:105EA0000E0180910F01909110016115710581051E
:105EB000910521F464E279ED8BE597E02DE133EF74
:105EC00041E050E00E94483149015A019B01AC0178
:105ED000A7EAB1E40E9467316B017C01ACEEB4EF3C
:105EE000A50194010E947531C60ED71EE81EF91E49
:105EF000F7FE06C081E0C81AD108E10880E8F80A78
:105F0000C0920D01D0920E01E0920F01F0921001AB
:105F1000C701B6019F77FF90EF90DF90CF90BF90C1
:105F2000AF909F908F90089560930D0170930E0134
:105F300080930F01909310010895FB01DC010590FF
:105F40000D920020E1F70895FC0105900020E9F78B
:105F5000809590958E0F9F1F0895BB274A3031F48E
:105F6000992322F4BDE2909581959F4F0C94EA2FDE
:105F7000BB272A3051F4992342F4BDE290958095D5
:105F8000709561957F4F8F4F9F4F0C94C82FBB2703
:105F9000FA01A62F6217710581059105330B30FBBD
:105FA00066F0AA27660F771F881F991FAA1FA217DE
:105FB00010F0A21B63953850A9F7A05DAA3308F032
:105FC000A95DA19336F7B111B1931082CA010C9467
:105FD0000330BB27FB015527AA27880F991FAA1F4B
:105FE000A41710F0A41B83955051B9F7A05DAA33F4
:105FF00008F0A95DA193009779F7B111B1931192BF
:10600000CB010C940330DC01FC01672F71917723E5
:10601000E1F7329704C07C916D9370836291AE1763
:10602000BF07C8F30895E89409C097FB3EF4909524
:106030008095709561957F4F8F4F9F4F9923A9F061
:10604000F92F96E9BB279395F695879577956795F0
:10605000B795F111F8CFFAF4BB0F11F460FF1BC034
:106060006F5F7F4F8F4F9F4F16C0882311F096E9C7
:1060700011C0772321F09EE8872F762F05C0662375
:1060800071F096E8862F70E060E02AF09A95660F2E
:10609000771F881FDAF7880F9695879597F90895E7
:1060A000990F0008550FAA0BE0E8FEEF1616170629
:1060B000E807F907C0F012161306E407F50798F091
:1060C000621B730B840B950B39F40A2661F0232BAA
:1060D000242B252B21F408950A2609F4A140A69526
:1060E0008FEF811D811D08950E9487300C94F83038
:1060F0000E94EA3038F00E94F13020F0952311F030
:106100000C94E1300C94E73011240C942C310E9453
:10611000093170F3959FC1F3950F50E0551F629FB1
:10612000F001729FBB27F00DB11D639FAA27F00DF0
:10613000B11DAA1F649F6627B00DA11D661F829F17
:106140002227B00DA11D621F739FB00DA11D621FFC
:10615000839FA00D611D221F749F3327A00D611D19
:10616000231F849F600D211D822F762F6A2F1124FB
:106170009F5750409AF0F1F088234AF0EE0FFF1F2E
:10618000BB1F661F771F881F91505040A9F79E3F85
:10619000510580F00C94E1300C942C315F3FE4F316
:1061A000983ED4F3869577956795B795F795E795DB
:1061B0009F5FC1F7FE2B880F911D9695879597F9E4
:1061C000089597F99F6780E870E060E008959FEF79
:1061D00080EC089500240A9416161706180609067E
:1061E000089500240A94121613061406050608954D
:1061F000092E0394000C11F4882352F0BB0F40F4D5
:10620000BF2B11F460FF04C06F5F7F4F8F4F9F4F14
:10621000089557FD9058440F551F59F05F3F71F096
:106220004795880F97FB991F61F09F3F79F08795FD
:106230000895121613061406551FF2CF4695F1DF86
:1062400008C0161617061806991FF1CF8695710516
:10625000610508940895E894BB2766277727CB014A
:1062600097F90895F999FECF92BD81BDF89A9927C3
:1062700080B50895262FF999FECF1FBA92BD81BD32
:1062800020BD0FB6F894FA9AF99A0FBE01960895B8
:10629000052E97FB1EF400940E945F3157FD07D036
:1062A0000E94B13107FC03D04EF40C945F3150953D
:1062B0004095309521953F4F4F4F5F4F08959095F2
:1062C0008095709561957F4F8F4F9F4F08950E94E5
:1062D000D331A59F900DB49F900DA49F800D911D6B
:1062E00011240895B7FF0C9467310E946731821B17
:1062F000930B08952F923F924F925F926F927F92ED
:106300008F929F92AF92BF92CF92DF92EF92FF92C5
:106310000F931F93CF93DF93CDB7DEB7CA1BDB0B71
:106320000FB6F894DEBF0FBECDBF09942A88398816
:1063300048885F846E847D848C849B84AA84B9841D
:10634000C884DF80EE80FD800C811B81AA81B98129
:10635000CE0FD11D0FB6F894DEBF0FBECDBFED013D
:106360000895A1E21A2EAA1BBB1BFD010DC0AA1F96
:10637000BB1FEE1FFF1FA217B307E407F50720F0AE
:10638000A21BB30BE40BF50B661F771F881F991F29
:106390001A9469F760957095809590959B01AC0172
:1063A000BD01CF010895A29FB001B39FC001A39F7B
:1063B000700D811D1124911DB29F700D811D11243E
:1063C000911D08955058BB27AA270E94FA310C94BA
:1063D000F8300E94EA3038F00E94F13020F039F4B1
:1063E0009F3F19F426F40C94E7300EF4E095E7FB98
:1063F0000C94E130E92F0E94093158F3BA17620773
:1064000073078407950720F079F4A6F50C942B31D7
:106410000EF4E0950B2EBA2FA02D0B01B9019001BF
:106420000C01CA01A0011124FF27591B99F0593F03
:1064300050F4503E68F11A16F040A22F232F342F4B
:106440004427585FF3CF469537952795A795F04099
:106450005395C9F77EF41F16BA0B620B730B840BAE
:10646000BAF09150A1F0FF0FBB1F661F771F881F66
:10647000C2F70EC0BA0F621F731F841F48F48795BE
:1064800077956795B795F7959E3F08F0B0CF9395B0
:10649000880F08F09927EE0F9795879508950E9429
:1064A00063320C94F8300E94F13058F00E94EA30C8
:1064B00040F029F45F3F29F00C94E13051110C9425
:1064C0002C310C94E7300E94093168F39923B1F321
:1064D000552391F3951B550BBB27AA27621773070A
:1064E000840738F09F5F5F4F220F331F441FAA1F9E
:1064F000A9F335D00E2E3AF0E0E832D0915050405A
:10650000E695001CCAF72BD0FE2F29D0660F771F07
:10651000881FBB1F261737074807AB07B0E809F0ED
:10652000BB0B802DBF01FF2793585F4F3AF09E3F72
:10653000510578F00C94E1300C942C315F3FE4F37A
:10654000983ED4F3869577956795B795F7959F5FB5
:10655000C9F7880F911D9695879597F90895E1E001
:10656000660F771F881FBB1F621773078407BA0760
:1065700020F0621B730B840BBA0BEE1F88F7E095BB
:1065800008950E94C8326894B1110C942C3108957A
:106590000E94113188F09F5798F0B92F9927B75171
:1065A000B0F0E1F0660F771F881F991F1AF0BA95B7
:1065B000C9F714C0B13091F00E942B31B1E00895B9
:1065C0000C942B31672F782F8827B85F39F0B93FAB
:1065D000CCF3869577956795B395D9F73EF490956A
:1065E0008095709561957F4F8F4F9F4F08950E94C2
:1065F000373390F09F3748F4911116F00C942C31FA
:1066000060E070E080E89FEB089526F41B16611DA2
:10661000711D811D0C940E330C942933882371F461
:10662000772321F09850872B762F07C0662311F42B
:1066300099270DC09051862B70E060E02AF09A9562
:10664000660F771F881FDAF7880F9695879597F959
:1066500008959F3F31F0915020F487957795679585
:10666000B795880F911D9695879597F908950E9483
:106670001131A0F0BEE7B91788F4BB279F3860F44A
:106680001616B11D672F782F8827985FF7CF86954C
:1066900077956795B11D93959639C8F308950E9433
:1066A000503008F48FEF089519F416F40C94E73085
:1066B0000C9429330E941131B8F39923C9F3B6F32E
:1066C0009F57550B87FF0E949A330024A0E640EAAB
:1066D000900180585695979528F4805C660F771F37
:1066E000881F20F026173707480730F4621B730B0A
:1066F000840B202931294A2BA6951794079420252D
:1067000031254A2758F7660F771F881F20F0261774
:106710003707480730F4620B730B840B200D311DD3
:10672000411DA09581F7B901842F9158880F969546
:106730008795089591505040660F771F881FD2F7B4
:106740000895DB018F939F930E946731BF91AF91B2
:10675000A29F800D911DA39F900DB29F900D1124BB
:106760000895EE0FFF1F0590F491E02D09940F930B
:106770001F93CF93DF938230910510F482E090E075
:10678000E0919E07F0919F0730E020E0B0E0A0E0AC
:10679000309799F42115310509F44AC0281B390BAB
:1067A00024303105D8F58A819B816115710589F105
:1067B000FB0193838283FE0111C0408151810281DC
:1067C000138148175907E0F04817590799F41097B3
:1067D00061F012960C93129713961C933296CF0188
:1067E000DF91CF911F910F91089500939E07109311
:1067F0009F07F4CF2115310551F04217530738F0A8
:10680000A901DB019A01BD01DF01F801C1CFEF0150
:10681000F9CF90939F0780939E07CDCFFE01E20FA3
:10682000F31F819391932250310939832883D7CF65
:1068300020919C0730919D07232B41F42091130157
:106840003091140130939D0720939C0720911101F2
:10685000309112012115310541F42DB73EB7409119
:10686000150150911601241B350BE0919C07F09106
:106870009D07E217F307A0F42E1B3F0B28173907DB
:1068800078F0AC014E5F5F4F2417350748F04E0F8C
:106890005F1F50939D0740939C07819391939FCFD7
:1068A000F0E0E0E09CCFCF93DF930097E9F0FC01AC
:1068B000329713821282A0919E07B0919F07ED013B
:1068C00030E020E01097A1F420813181820F931FE6
:1068D00020919C0730919D072817390709F061C066
:1068E000F0939D07E0939C07DF91CF910895EA0113
:1068F000CE17DF07E8F54A815B819E0141155105FE
:10690000B1F7E901FB83EA8349915991C40FD51F7F
:10691000EC17FD0761F4808191810296840F951F29
:10692000E90199838883828193819B838A83F0E044
:10693000E0E012968D919C9113970097B9F52D91F7
:106940003C911197CD010296820F931F20919C07D5
:1069500030919D072817390739F6309751F5109275
:106960009F0710929E07B0939D07A0939C07BCCFF2
:10697000D383C28340815181840F951FC817D907E3
:1069800061F44E5F5F4F88819981480F591F518391
:1069900040838A819B81938382832115310509F08D
:1069A000B0CFF0939F07E0939E079ECFFD01DC01DF
:1069B000C0CF13821282D7CFB0E0A0E0E2EEF4E3C2
:1069C0000C947C318C01009751F4CB010E94B733B9
:1069D0008C01C801CDB7DEB7E0E10C949831FC0121
:1069E000E60FF71F9C0122503109E217F30708F464
:1069F0009DC0D901CD91DC911197C617D70798F0AA
:106A0000C530D10530F3CE0104978617970708F3F8
:106A1000C61BD70B2297C193D1936D937C93CF0163
:106A20000E945334D6CF5B01AC1ABD0A4C018C0EC8
:106A30009D1EA0919E07B0919F07512C412CF12CD7
:106A4000E12C109731F580919C0790919D07881556
:106A5000990509F05CC04616570608F058C08091A9
:106A6000110190911201009741F48DB79EB74091AA
:106A7000150150911601841B950BE817F90708F0D2
:106A800055C0F0939D07E0939C07F90171836083E3
:106A9000A0CF8D919C91119712966C90129713969E
:106AA0007C901397A815B90559F56C0142E0C40E06
:106AB000D11CCA14DB0420F1AC014A195B09DA01CC
:106AC0001296159780F06282738251834083D901B8
:106AD0006D937C93E114F10471F0D7011396FC934C
:106AE000EE93129776CF22968C0F9D1FF90191831A
:106AF0008083F301EFCFF0939F07E0939E0769CF68
:106B00004816590608F42C017D01D3019ACFCB0118
:106B10000E94B7337C01009749F0AE01B8010E9492
:106B20009935C8010E945334870153CF10E000E02B
:106B300050CFFB01DC0102C001900D92415050404A
:106B4000D8F70895FB01DC0101900D920020E1F7D8
:106B5000089517E0C0EBD7E004C0FE010E94B133F6
:0C6B60002196C13BD107C9F7F894FFCF84
:106B6C0010FFFFFFFF00E10000000000000100002B
:106B7C00000000A007800000C18081000000000020
:106B8C000000F40B5F0D150C0A0C5B0C190C370C88
:106B9C00000000004F12C90E8813E40D0000000025
:106BAC000112C90E8813E40D00000000C910C90EB3
:106BBC008813E40D596F7520656174206974206128
:106BCC006C6C2062757400666F7267657420746FEC
:106BDC0020627275736820796F75720074656574C4
:106BEC00682E205468657920616C6C20726F74007B
:106BFC00616E6420796F752063616E277420656106
:106C0C007400736F6C696420666F6F6420616E79B9
:106C1C006D6F72652E002020204A7573742073618D
:106C2C0079206E6F0020202020746F2063616E64C9
:106C3C00792E00202047616D65206F7665722100EA
:106C4C002020596F75722073636F72653A20002093
:106C5C00206F7574206F66203130302E00696E20E5
:106C6C0061206C756E636820626F7820696E0074A9
:106C7C0068652073756277617921212100546865FC
:106C8C00206D61726B657420686173006265656E5E
:106C9C0020666C6F6F646564207769746800636844
:106CAC0065617020686F6D656D616465004165722A
:066CBC006F2121212100DF
:00000001FF
